:020000040800F2
:10000000C04B00208102000889470008933F000888
:100010004D460008410B0008BD5E000800000000CE
:10002000000000000000000000000000A101000826
:10003000BF0B000800000000FD0100082D50000863
:100040009B0200089B0200089B0200089B0200081C
:100050009B0200089B0200089B0200089B0200080C
:100060009B0200089B0200089B020008450B000849
:10007000510B0008650B0008790B0008850B000880
:100080009B0200089B0200089B0200089B020008DC
:100090009B0200089B0200089B0200089B020008CC
:1000A0009B0200089B020008E9500008C9500008A4
:1000B0009B02000800000000000000009B020008F6
:1000C0009B0200089B0200089B0200089B0200089C
:1000D0009B020008B95C00089B0200089B02000814
:1000E0009B0200089B0200080000000000000000C6
:1000F0000000000000000000000000000000000000
:10010000000000009B020008000000009B020008A5
:100110000000000000000000F55000089B020008ED
:100120009B0200089B0200089B0200089B0200083B
:100130009B0200080000000000000000000000001A
:100140009B0200089B0200089B02000800000000C0
:100150009B0200089B0200089B0200089B0200080B
:100160009B0200089B0200089B02000800000000A0
:100170009B0200089B020008000000000000000035
:100180009B0200089B0200089B020008DFF80CD0CD
:1001900000F01EFB00480047F5680008C04B002037
:1001A0002C4B1968086800F05AB880F30988BFF32F
:1001B0006F8F4FF0000080F311887047000000003F
:1001C00008480068006880F308884FF0000080F35A
:1001D000148862B661B6BFF34F8FBFF36F8F00DF35
:1001E00000BF00BF08ED00E0DFF80C00016841F43B
:1001F00070010160704700BF88ED00E0EFF30980F7
:10020000BFF36F8F134B1A681EF0100F08BF20ED5D
:10021000108A20E9F04F106009B44FF0500080F3CD
:100220001188BFF34F8FBFF36F8F07F09DFC4FF026
:10023000000080F3118809BC1968086800F014B840
:100240001EF0100F08BF00F014B880F30988BFF348
:100250006F8F7047A4010020EFF30580704730C80E
:10026000B0E8C04FFFF7A1BF30C8B0E8C04FFFF7FC
:10027000E7BFB0EC088AB0EC08CAFFF7E6BF0000A1
:100280000648804706480047FEE7FEE7FEE7FEE730
:10029000FEE7FEE7FEE7FEE7FEE7FEE7B9500008EF
:1002A0008D0100082DE9F05F0546002092469B462F
:1002B00088460646814640241BE02846414647467C
:1002C000224600F093F853465A46C01A914110D383
:1002D00011461846224600F07AF82D1A67EB0108FD
:1002E0004F4622460120002100F071F817EB00096B
:1002F0004E41201EA4F10104DFDC484631462A4667
:10030000434600F000B830BCBDE8C09F40EA01039E
:100310009B0703D009E008C9121F08C0042AFAD2BB
:1003200003E011F8013B00F8013B521EF9D270477F
:10033000D2B201E000F8012B491EFBD27047002227
:10034000F6E710B513460A4604461946FFF7F0FFD4
:10035000204610BD421C10F8011B0029FBD1801A59
:10036000704730B504460020034600E05B1C934212
:1003700003D2E05CCD5C401BF8D030BD00F0004201
:1003800030F000400AD0C10D01F56071C0F31600D5
:1003900042EA0151C208400711437047002001465C
:1003A000704730B50B46014600202022012409E0A9
:1003B00021FA02F59D4205D303FA02F5491B04FA1E
:1003C00002F52844151EA2F10102F1DC30BD202AFD
:1003D00004DB203A00FA02F1002070479140C2F19C
:1003E000200320FA03F3194390407047202A04DBCE
:1003F000203A21FA02F00021704721FA02F3D0409E
:10040000C2F12002914008431946704710B54100DF
:100410000CD0C0F3C751962908DC7E2909DC06DB25
:10042000410204D000F0004040F07E5010BD00209A
:1004300010BDC1F19604C4F1200100FA01F1E040C1
:1004400000F0EAF9A04010BD2DE9FE4F804681EA98
:100450000300C00F0C46009021F0004123F000453E
:10046000B8EB0200A94105D24046214690461C4601
:100470000B46024623F00040104347D0270DC7F338
:100480000A00C3F30A510290401A019040286BDA27
:10049000C3F3130040F4801B0098924620B1002360
:1004A000D2EB030A63EB0B0B01985946C0F14002F3
:1004B0005046FFF78CFF06460D4650465946019AB6
:1004C00000F098F910EB08006141002487EA11520E
:1004D00084EAE7731A4340D0009A62B3019A012A72
:1004E0004FEA075215DC001B61EB02014FF000429E
:1004F00002EA0752CDE90042001C41F58011324664
:100500002B4600F0CFF903B000F045B84046214635
:10051000F9E7001B61EB0201001C41F58013001894
:100520005B412018A2F5001747EB030140EAD570A4
:10053000B6196D4111E06D084FEA360645EAC075FF
:100540004FEA0752001B61EB0201001C41F58011CC
:1005500049084FEA30000019514132462B4603B09A
:1005600000F01CB800F08FB9009801224000002371
:10057000D0EB020263EBE073009821464FEAE0748F
:10058000B8EB000061EB0401E9E783F000435BE7AF
:1005900081F0004158E730BCBDE8C08F30BCBDE8F9
:1005A000C04FFFF7DFBF2DE9FE4F81EA030404F0DF
:1005B000004421F0004100944FF0000B23F0004371
:1005C00050EA01045ED052EA03045BD0C3F30A543C
:1005D000C1F30A552C44A4F2F3340194A0FB025455
:1005E000C1F3130141F48011C3F3130343F48013E7
:1005F00001FB024400FB034E840A970A44EA81543B
:1006000047EA8357A4FB076802958D0A05FB078517
:100610004FEA932C04FB0C542705029D4FEA065821
:1006200047EA1637B5EB08056EEB070C870E920EFE
:1006300047EA811742EA8312A7FB0201B6EB0B01DE
:1006400064EB00042B0D43EA0C335E1844EB1C50A2
:10065000DA465146E7FB0201C5F313044FEA0B33B8
:1006600043EA14534FEA0432019C43EA0603A4F11F
:100670000C040294009CCDE900B400F013F903B01F
:1006800000F003B800200146F9E730BCBDE8C08F98
:100690002DE9F04D81EA030404F0004B21F0004500
:1006A00014464FF0000A23F0004150EA050220D022
:1006B00054EA01021DD0C5F30A570246C5F31303DD
:1006C000C1F31300C1F30A5640F4801543F48013BC
:1006D000A7EB0608101BD64608F2FD3873EB0500A1
:1006E00002D308F1010801E092185B41B8F1000F54
:1006F00003DA00200146BDE8F08D00204FF48011A0
:10070000064684460EE0171B73EB050705D3121B44
:1007100063EB050306434CEA010C49084FEA30003D
:1007200092185B4150EA0107EDD152EA030012D062
:1007300082EA040083EA0501084305D0101BAB419F
:1007400006D20122002306E000224FF0004302E01F
:100750006FF0010253101AEB06004CEB085110EB3E
:100760000A0041EB0B01BDE8F04D00F08CB8C1F37D
:100770000A52C1F3130140F2FF3341F480119A424F
:1007800002DA00200146704740F233439A42A2F257
:10079000334202DC5242FFF729BEFFF718BE0000C9
:1007A00030B5041E71F1000404DB4FF000444042F8
:1007B00064EB0101141E73F1000405DB1C464FF0CD
:1007C0000043524263EB0403994208BF904230BD9C
:1007D000064C074D06E0E06840F0010394E807008E
:1007E00098471034AC42F6D3FFF7D4FC08880008D1
:1007F00028880008202A06DBCB17203A41FA02F0AD
:1008000043EAE07306E041FA02F3D040C2F120026D
:1008100091400843194670470029A8BF7047401C03
:10082000490008BF20F00100704710B4B0FA80FC06
:1008300000FA0CF050EA010404BF10BC704749B143
:10084000CCF1200421FA04F411FA0CF118BF0121B3
:1008500021430843A3EB0C01CB1D4FEA00614FEA93
:10086000102042BF002010BC704700EBC350104462
:100870000029A4BF10BC7047401C490008BF20F0ED
:10088000010010BC704710B5141E73F1000408DAA3
:10089000401C41F1000192185B411A4301D120F044
:1008A000010010BD2DE9F04D92469B4611B1B1FA01
:1008B00081F202E0B0FA80F220329046FFF787FD25
:1008C00004460F4640EA0A0041EA0B0153465A46E5
:1008D000084313D0114653EA010019D0C8F1400271
:1008E0005046FFF783FD05460E46504659464246A0
:1008F000FFF76DFD084305D0012004E0204639468E
:10090000BDE8F08D0020054346EAE0762C433743EE
:100910000A986305E40AA0EB08000022FD0A44EAF5
:1009200047540A3002D500200146E9E701051019B5
:100930006941DDE9084500196941BDE8F04DA2E7CC
:1009400070B58C1810F8015B15F0070301D110F891
:10095000013B2A1106D110F8012B03E010F8016BBE
:1009600001F8016B5B1EF9D12B0705D40023521E41
:100970000DD401F8013BFAE710F8013BCB1A921CA9
:1009800003E013F8015B01F8015B521EF9D5A142A7
:10099000D8D3002070BD10B5846A616D11F0500F7E
:1009A00006D0616DC90625D5204600F07EFC10BD3D
:1009B000606D40F40070606520680168090716D515
:1009C00003F05FFB78B12068C068800400280ADB70
:1009D000606D20F480706065606DC00403D4606D4C
:1009E00040F001006065204600F05DFC10BDC0686D
:1009F0008007EBE7E16C496BBDE81040084710B594
:100A0000806A416D41F040014165816D41F0040112
:100A1000816500F04AFC10BD10B5806A00F044FC0E
:100A200010BD000070B50446006881688268C1F39B
:100A3000400112F0010F28D039BB816801F00D018F
:100A4000012914D18168124A1140891C81602168F2
:100A50000320086001F0D8F9054612E001F0D4F94E
:100A6000401B02280DD920688068C00709D0606D3E
:100A700040F010006065A06D40F00100A06501200D
:100A800070BD20688068C007E8D1002070BD0000FC
:100A9000C0FFFF7FF8B50446002000902068816801
:100AA00011F0010F41D18168214A11422ED1816894
:100AB000D5432940491C81601E48806800F0E070E1
:100AC00000020DD51C481D490068B0FBF1F0401C28
:100AD00000EB4000800000E0401E00900028FBD1A9
:100AE00001F092F906461BE0816811F0010F03D175
:100AF00081682940491C816001F086F9801B022829
:100B00000ED920680068C043C00709D0606D40F06E
:100B100010006065A06D40F00100A0650120F8BDE7
:100B200020680168C943C907DED10020F8BD000074
:100B30003F0000800003045074000020400D0300BB
:100B4000FEE70000014800F0F3BD0000380D002072
:100B500010B5034800F0ECFDBDE8104003F08EBE78
:100B6000040F002010B5034800F0E2FDBDE810407E
:100B700003F084BE4C0F0020014800F0D9BD0000F6
:100B8000E4100020014800F0D3BD00009C100020BC
:100B900030B590F8444004F01C050124AC40056CCD
:100BA0006C60046863608368102B036803D09960ED
:100BB0000068C26030BD9A600068C16030BD704797
:100BC00072B6FEE7144A117F1448012901D00329A7
:100BD0000FD1036823F400730360036843F40063D8
:100BE0000360036823F400630360036843F4007345
:100BF0000360022901D003290BD1016841F480511F
:100C00000160016821F480510160016841F4806154
:100C1000016000201077704754000020002002403F
:100C2000C107054803D0416941F0040141614169B0
:100C300041F48031416170470020024008494A690F
:100C4000C0B222F47E7242EAC0004861486940F0B6
:100C500002004861486940F48030486170470000F4
:100C600000200240054910B54C6944F001044C6174
:100C70000260BFF36F8F436010BD00000020024090
:100C8000094A10B55469402344F480245461EFF3B9
:100C9000108272B610C910C05B1E13F0FF03F9D1A9
:100CA00082F3108810BD00000020024070B5054698
:100CB00001F0AAF80646134C08E0681C06D001F0C3
:100CC000A3F8801BA84201D3032070BD2069C00394
:100CD000F3D420690C4908400CD00C494A680243FF
:100CE0004A60810F01D0A169A161810000D020611B
:100CF000012070BD2069C00701D0012020610020C3
:100D000070BD000000200240FAC302005400002021
:100D100070B586B00C00054628D01548854225D808
:100D20000026049600F0CAFE1248816941F0404155
:100D300081614CF2FA3101612846009600F01CF8FE
:100D40000190284600F026F8029005EB8400401E32
:100D500000F020F80299401A401C039004A968464C
:100D600000F0DCFD002801D000F048FE06B070BDA8
:100D700000000408002002400449096804494FF0BB
:100D800001000968CA431204120C704700000140B8
:100D9000E075FF1F0E4910B509684FF48024CB435E
:100DA0001A04120C0AD00A045FEA921202F10062DD
:100DB000824205D9A0F10060C00A10BD2246F5E7C5
:100DC0001A04120C01D009048C09001BF2E7000080
:100DD000E075FF1F2DE9F04117460D46044600F06F
:100DE0006DFE0F48844216D2002609E0D5E90023A3
:100DF0002146002000F00CFE68B908340835761C46
:100E0000B6EB570FF2D3F80705D0636821460020F0
:100E10002A6800F0FDFDBDE8F04100F0EFBD0000E4
:100E200000000408F8B500260446009690F850002B
:100E30000D4601280BD0012084F850002046FFF712
:100E4000F1FD0100606D04D040F010002BE00220A5
:100E5000F8BD20F4885040F0020060652068826888
:100E6000134B1A4005F080431A4342F0004282605F
:100E70004FF4912320680EE0009A521C00929A428F
:100E800009D3606D20F0020040F01000606584F826
:100E900050600120F8BD8268D20FEDD1606D20F066
:100EA000020040F00100606584F850600846F8BD1B
:100EB000C0FFFF3F2DE9F84F00270446009790F848
:100EC0005000DFF8B0930D46B846012811D0012636
:100ED00084F85060206803F0D0F860B1606D40F095
:100EE000200060655FF0010784F85080384600F00C
:100EF000D7B90220FBE769680C20052912D802291E
:100F000007D0032907D0042907D0052907D00621D7
:100F100007E0686006E0122103E0182101E04FF4C9
:100F200080716960D5E90021236800EA91101844B6
:100F3000036B01F01F014FF01F0C0CFA01FCC2F310
:100F4000846223EA0C038A4013430363206803F09E
:100F500094F88246206803F08CF85AEA00001DD10C
:100F6000AA682968206803F094F820686969C26853
:100F7000C2F3C102520091402A69042A0FD000EB4B
:100F800082002B68026EDFF8F0C203F0F84302EA39
:100F90000C020B431A4342F00041016672E000214B
:100FA00003F061F8400320684FF0000172D003F0B5
:100FB0005AF890FAA0F0B0FA80F1286842036ED097
:100FC00090FAA0F0B0FA80F0814204D100221146DC
:100FD000206803F06DF80121206803F044F8400315
:100FE00020684FF001015DD003F03DF890FAA0F0C9
:100FF000B0FA80F12868420359D090FAA0F0B0FA14
:1010000080F0814204D100220121206803F050F8D1
:101010000221206803F027F8400320684FF0020106
:1010200048D003F020F890FAA0F0B0FA80F12868D8
:10103000420344D090FAA0F0B0FA80F0814204D18B
:1010400000220221206803F033F80321206803F016
:101050000AF8400320684FF0030133D003F003F88F
:1010600090FAA0F0B0FA80F1286842032FD090FAED
:10107000A0F0B0FA80F0814204D100220321206860
:1010800003F016F82068816811F0010F22D0ABE060
:1010900000E004E002F0E7FFC0F384618DE7C0F3F5
:1010A000846091E702F0DFFFC0F38461A2E7C0F340
:1010B0008460A6E702F0D7FFC0F38461B7E7C0F30E
:1010C0008460BBE702F0CFFFC0F38461CCE7C0F3DC
:1010D0008460D0E72A7B296850F8B03FC1F3120C36
:1010E00023EA0C0302F0180C644A22FA0CF20A40BC
:1010F00013430360E968494576D1286841031BD052
:1011000090FAA0F1B1FA81F1491C01F01F010929FF
:101110004FEA403131D8002911D090FAA0F1B1FA4C
:1011200081F100BF01F1010101F01F0106FA01F692
:1011300008D1C0F3846109E0C0F38461E4E7C0F33F
:101140008461EFE790FAA0F1B1FA81F101F10101B8
:1011500001F01F0146EA816102D1C0F3846003E01F
:1011600090FAA0F0B0FA80F000F1010000F01F004A
:1011700000EB400041EA005132E000290ED090FA25
:10118000A0F1B1FA81F100BF01F1010101F01F01ED
:1011900006FA01F605D1C0F3846106E0C0F384616C
:1011A000F2E790FAA0F1B1FA81F101F1010101F049
:1011B0001F0146EA816102D1C0F3846003E090FA26
:1011C000A0F0B0FA80F000F1010000F01F002C4AFE
:1011D00000EB400002EB005041EA000141F00071D9
:1011E000AA68206802F055FF26482A6802423FF4A8
:1011F0007BAE25488168254D254B01F0E071AA4260
:101200001BD10D0219D422689A427FF46DAE826818
:1012100041F4000122F0E0720A4382601D481E4939
:101220000068B0FBF1F0401C00EB4000800000E0E3
:10123000401E00900028FBD156E6184DAA4207D167
:10124000CD0105D422689A42F6D141F080710AE0BE
:101250006FF00045EA42EFD14A02EDD422689A428B
:10126000EAD141F48001826822F0E0720A43826090
:101270003AE6000000007F4000F0FF03FFFF070098
:10128000000020FE0000088000030450000052C748
:101290000000045074000020400D0300000084CBC7
:1012A00018BCBDE8E08F704770477047F8B54FF045
:1012B000000504002E46009502D0606D10B107E0D5
:1012C0000120F8BD204600F0C9F8A66584F85060FA
:1012D00020688168C1F3407119B18168574A114093
:1012E000816020688168C1F3007189B98168544ABE
:1012F000114041F080518160524853490068B0FB71
:10130000F1F04000801C00E0401E00900028FBD15E
:1013100020688168C1F3007141B9616D41F010012D
:101320006165A16D41F00101A165012502F0A5FEF5
:10133000616D01F010010143606D05D040F01000B7
:10134000606501252846F8BD20F4807040F0020059
:1013500060652068806810F0010F0BD13B48806801
:1013600010F0010F06D13A486168826822F47C12BD
:101370000A438260E168606B627E0843A16841EACB
:101380004231084394F8201040EA0140012904D179
:10139000A18C304A02EB41410843A16A29B101F412
:1013A0007071E26A014342EA01002268D1682A4B67
:1013B00019400143D160206802F05FFE06462068B4
:1013C00002F057FE304315D1207E94F83010800390
:1013D00040EA41022068C16844F202039943114384
:1013E000C16094F8380001280CD02068016921F010
:1013F00001010161206901282068016B21F00F01C2
:1014000011D013E0D4E90F010843D4E911121143BC
:10141000084321680A6940F2FC739A43104340F084
:1014200001000861E6E7E269521E11430163606D45
:1014300020F0020040F00100606583E7C0FFFF5F1D
:10144000C0FFFF7F74000020400D03000000045027
:10145000000304500000FEFF07C0F0FFF0B59DB090
:101460000646142117A8FEF76AFF5C216846FEF7BE
:1014700066FF2F493068884258D14FF48040009071
:101480008003149002240120CDE90140082003903C
:101490000720CDE904048801CDE90640684600F044
:1014A000B3FE08B1FFF78CFB2249C86C40F4005032
:1014B000C864C86C00F400501C90C86C40F0010077
:1014C000C864C86C00F001001C90C86C40F00200B9
:1014D000C864C86C002500F002001C90F0200B27A7
:1014E0001995CDE9170717A94FF0904000F09CFB24
:1014F0001995CDE9174717A90F4800F095FB104C37
:101500000E48C4E900058020A560C4E903504000EE
:1015100060618000A0612020C4E90705204600F03A
:1015200065F908B1FFF74CFBF464A6621DB0F0BD8D
:10153000000004500010024000040048080002406F
:10154000380D002070B5044615460E46006802F0BE
:1015500094FDE0BB94F85000012842D0012084F8AB
:1015600050002046FFF796FA002110B184F8501081
:1015700070BD606D40F60162904340F4807060651C
:10158000606DC00404D5A06D20F00600A06500E0E9
:10159000A165E26C1448D062E26C14481063E26CFE
:1015A0001348506322681C20106084F85010206893
:1015B000416841F0100141602068C16841F00101BB
:1015C000C16021682B4632464031E06C00E008E003
:1015D00000F06CF921688A68064B1A40121D8A6077
:1015E00070BD022070BD000097090008190A0008AC
:1015F000FF090008C0FFFF7F10B590F825100022FA
:10160000022905D00421C16380F82420012010BDE7
:1016100001680B6823F00E030B6001680B6823F070
:1016200001030B6090F84410046C01F01C030121CD
:1016300001FA03F3636080F8251080F82420104637
:1016400010BD10B590F825100024022903D0042104
:10165000C16301241AE001680A6822F00E020A60E0
:1016600001680A6822F001020A6090F84410036CD5
:1016700001F01C02012101FA02F25A6080F82510E3
:10168000002180F82410816B01B18847204610BDED
:1016900030B590B101680A6822F001020A60204C5E
:1016A000036814211F4AA34209D21F4C1C44B4FBF7
:1016B000F1F18900C0E910210BE0012030BD184C88
:1016C00064421C44B4FBF1F18900416414490839B7
:1016D00001640021196090F8443003F01C040123D8
:1016E000A340046C6360046C0F23944202D152F84F
:1016F000A84F02E00A4AA032146890F8445005F05E
:101700001C05AB409C431460C1620163416381636B
:10171000C16380F8251080F82410002030BD00003F
:101720000804024000000240F8FFFDBFC06B704794
:10173000F0B4016C0C6801680D6890F8442002F068
:101740001C06042202FA06F3234211D06B070FD5C0
:101750000B689B0603D40B6823F004030B6090F81E
:10176000441001F01C018A40016C4A60016B1DE0CD
:10177000022303FA06F727424FF0000C4FF0010254
:1017800018D0AF0716D50C68A40605D40C6824F051
:101790000A040C6080F8252090F8441001F01C0128
:1017A0008B40016C4B6080F824C0C16A00291AD0BC
:1017B000F0BC08470823B340234214D02B0712D5AE
:1017C0000B6823F00E030B6090F84410036C01F0DB
:1017D0001C0102FA01F15960C26380F8252080F8EB
:1017E00024C0416BE2E7F0BC7047000070B568B1FF
:1017F0002B4C036814212B4AA34209D22A4C1C44C7
:10180000B4FBF1F18900C0E910210BE0012070BDAB
:10181000234C64421C44B4FBF1F18900416420492B
:1018200008390164022180F825101C6847F6F07120
:101830008C43D0E902152943D0E9045635432943A6
:1018400085692943C5692943056A294321431960EC
:101850008168B1F5804F19D0036C0F21934202D1FA
:1018600052F8A83F02E00E4AA032136890F84440B4
:1018700004F01C04A1408B43136090F8443041688D
:1018800003F01C0399401368194311600021C163E0
:10189000012280F8252080F82410084670BD000041
:1018A0000804024000000240F8FFFDBF70B5044686
:1018B00090F82400002501280CD0012084F8240091
:1018C00094F825600020012E06D084F8240002251B
:1018D000284670BD022070BD022684F82560E063B2
:1018E0002068066826F0010606602046FFF750F9DA
:1018F000206B00282068016802D041F00E0106E04C
:1019000021F0040101602068016841F00A010160D2
:101910002068016841F001010160D9E72DE9F05F1D
:10192000054632488946017801290CD001268046B7
:1019300006704CF2503B5846FFF7B8F907004FF0DD
:10194000000A03D04EE0022000F054B85146404651
:10195000C8F804A0264C226892050AD521684905DA
:1019600005D5216821F480612160032109E0067713
:1019700008E02268520504D5216821F480612160C5
:10198000022101772868012807D04FF0FF31C9F8FC
:10199000001040F2FA3BAE681DE06868FFF740F9BE
:1019A0005846FFF783F90746606920F0040060613C
:1019B00016E030466968FFF741F94CF25030FFF706
:1019C00075F90700606920EA0B00606102D0C9F870
:1019D000006005E0761CD5E902010844B042E8D871
:1019E000FFF7F0F888F800A03846ADE75400002073
:1019F0000020024030BCBDE8C09F000003484169A0
:101A000041F0004141610020704700000020024089
:101A10002DE9FF5F254C0646904620789A4601281E
:101A20000BD0012020704CF2503B5846FFF73EF996
:101A300007004FF0000904D02AE0022004B000F0B3
:101A400039B84846C4F80490194D2968490504D5A9
:101A5000286820F4806028600220207726B1012EBB
:101A600009D0022E07D00CE0424653460198FFF7FA
:101A7000F9F8012612E041460198FFF701F9022E1C
:101A80000AD05846FFF712F94FEA0007FFF79AF815
:101A900084F800903846D1E74FF480265846FFF787
:101AA00005F907466869B0436861EFE75400002014
:101AB0000020024030BCBDE8C09F00000649002065
:101AC0004A69002A07DA054A8A60054A8A60496934
:101AD000002900DA012070470020024023016745F9
:101AE000AB89EFCD2DE9F84F00230126DFF818C1AF
:101AF0000F2782E006FA03F414EA01027CD023F0F7
:101B000003056544AA46D5F808909D074FEA157E5F
:101B100007FA0EF505EA090B0095B0F1904F05D0D4
:101B20003A4DA84205D14FF0010816E04FF00008E9
:101B300013E0374DA84202D14FF002080DE0354DB9
:101B4000A84202D14FF0030807E0334DA84202D16A
:101B50004FF0040801E04FF0070808FA0EF8D845E6
:101B600026D1DFF8B880D8F8009029EA0209C8F831
:101B7000009008F10408D8F8009029EA0209C8F892
:101B80000090DFF8988008F10C08D8F8009029EA56
:101B90000209C8F80090A8F10408D8F8005095434D
:101BA000C8F80050009DDAF80820AA43CAF80820B7
:101BB000D0F800804FEA4309032202FA09F248EA0A
:101BC0000208C0F80080DD0800EB8505AA46D5F8BC
:101BD00020804FEA43794FEAD96907FA09F528EAE4
:101BE0000508CAF820808568954385604568A54347
:101BF0004560C4689443C4605B1C31FA03F27FF40F
:101C000079AF00F00DB8000000000140000400486A
:101C100000080048000C0048001000480004014083
:101C200018BCBDE8E08F00002DE9F04FDFF8AC9163
:101C300000230325A9F1040B85B04FF0010C0F27F9
:101C400009F1040AABF1040EBFE000BF0CFA03F681
:101C5000324075D00C7904F00304012C01D0022C21
:101C60001BD1846800945C0005FA04F80494009C7D
:101C700024EA08040094D1F80C80049C08FA04F8C3
:101C8000009C48EA0408C0F808804468B4430E7910
:101C9000C6F300169E40264346600C79E443A40731
:101CA0000AD0C4684FEA430805FA08F6B4438E68C0
:101CB00006FA08F62643C6600C7904F00304022CE9
:101CC00010D1DC0800EB84040294246A5E074FEA1A
:101CD000D66807FA08F6B4430E6906FA08F62643F2
:101CE000029C266204684FEA430805FA08F6B443EA
:101CF0000E7906F0030606FA08F6264306604C68DD
:101D000014F4403F60D0364C266E46F0010626663D
:101D1000246E23F0030604F001040094314C344493
:101D20000294A4689E074FEA167807FA08F6B443AF
:101D3000B0F1904F05D02C4EB04204D1012612E0F4
:101D400042E000260FE0294EB04201D102260AE00F
:101D5000274EB04201D1032605E0264EB04201D104
:101D6000042600E0072606FA08F62643029CA66031
:101D7000D9F800604C46D1F8048096435FEAC82841
:101D800000D516432660DAF800405646D1F80480A4
:101D900094435FEA882800D514433460DBF80040A0
:101DA0005E46D1F8048094435FEA883800D5144336
:101DB0003460DEF800407646D1F8048094435FEA50
:101DC000C83800D5144334605B1C0A6832FA03F447
:101DD0007FF43CAF05B000F00FB8000008040140EC
:101DE00000100240000001400004004800080048C4
:101DF000000C00480010004830BCBDE8C08F0AB19C
:101E000081617047816270470148806870470000B7
:101E10004800002090F84120202A24D190F840204A
:101E2000012A20D0012280F84020242280F841207D
:101E30000268136823F0010313600268136823F437
:101E400080531360026813680B43136001680A68CB
:101E500042F001020A60202180F84110002180F840
:101E60004010084670470220704790F84120202A11
:101E700022D190F84020012A1ED0012280F8402073
:101E8000242280F841200268136823F001031360C4
:101E90000268136823F4706343EA0121116001684A
:101EA0000A6842F001020A60202180F841100021F6
:101EB00080F84010084670470220704770B5040053
:101EC00004D094F84100002510B106E0012070BD57
:101ED00084F84050204600F04DF8242084F841005A
:101EE0002068016821F0010101606068216820F02C
:101EF000706008612068816821F400418160E068B9
:101F00000128A06807D040F4044021688860E06898
:101F1000022803D006E040F40040F6E721684FF4C1
:101F20000060486020684168114A114341602068A0
:101F3000C16821F40041C160D4E904010843A169EA
:101F400040EA01202168C860D4E9070108432168FC
:101F500008602068016841F001010160656420208B
:101F600084F84100256384F84250002070BD0000D1
:101F70000080000230B59DB00446142117A8FEF77A
:101F8000DEF95C216846FEF7DAF9174920688842D5
:101F900027D18020002500900D95684600F034F987
:101FA00008B1FEF70DFE114CE06C40F00200E06459
:101FB000E06C17A900F002001C904FF4C04017908D
:101FC0001220CDE918050420CDE91A500848FFF782
:101FD0002BFEA06D40F48000A065A06D00F4800091
:101FE0001C901DB030BD00000058004000100240A1
:101FF00000040048024881680278114481607047FB
:102000004800002010B50024032000F0AFF80F2096
:1020100000F008F808B1012401E000F04FF8204674
:1020200010BD000030B505461F4887B0816D41F0F6
:1020300010018165806D06A900F01000009001A8D4
:1020400000F0E2FA0498B0B100F0FEFA400017493F
:10205000174AB0FBF1F11748491E0260416040F297
:10206000E7320021C0E903218160816100F04CFE6C
:10207000040003D015E000F0E7FAE8E70D4800F0AF
:1020800019FF04000DD1362000F043F8102D07D2BF
:1020900000222946362000F049F80748056000E094
:1020A000012407B0204630BD0010024040420F001E
:1020B000001000402C1200204C0000200B4882B081
:1020C000016E41F001010166016E01F00101009114
:1020D000816D41F080518165806D002200F080505B
:1020E00000900F21901E02B000F020B800100240B6
:1020F00000280DDB00F01F02012191404009800003
:1021000000F1E020C0F88011BFF34F8FBFF36F8F55
:102110007047002809DB00F01F02012191404009AF
:10212000800000F1E020C0F800117047F0B40E4BC1
:102130001B680C46C3F30223C3F10705042D00D925
:102140000425191D072901D2002300E0DB1E01260A
:1021500006FA05F1491E214099409E40761E164020
:102160003143F0BC03F0BCBE0CED00E0064900F0CA
:10217000070208684FF6FF03184040EA0220034AAE
:1021800010430860704700000CED00E00000FA0505
:102190001649B0F5007F0868C0F3412009D0022835
:1021A00005D0086820F4C06040F48060086000201A
:1021B00070470128FBD0086820F4C06040F400702C
:1021C00008600B483222006850430A4AB0FBF2F024
:1021D000401C00E0401E4A69520501D50028F9D193
:1021E00048694005E3D503207047000000700040B7
:1021F0007400002040420F000248006800F4C060F4
:1022000070470000007000402DE9F84F0446002799
:102210000088A84D3E46000515D5606C60B1B0F54C
:10222000000F04D0B0F5400F2BD001270AE0E8687A
:1022300040F48030E86024E00021201D02F014FC0E
:1022400007001ED03E46206880033AD5A86D4FF0A7
:102250000008C00009D4A86D40F08050A865A86DA2
:102260004FF0010800F080500090DFF84CA2DAF83F
:10227000001041F48071CAF80010FFF7C5FD8146D7
:1022800010E0D5F88800616C20F440000843C5F8E0
:102290008800D8E7FFF7B8FDA0EB0900022801D9B4
:1022A000032705E0DAF80000C005F3D5002F7DD044
:1022B0004FEA0706B8F1000F03D0A86D20F0805058
:1022C000A8652078C00707D0D5F88800216A20F0DB
:1022D00003000843C5F888002078800707D5D5F8A3
:1022E0008800616A20F00C000843C5F88800207857
:1022F000400707D5D5F88800A16A20F030000843D0
:10230000C5F888002078800607D5D5F88800E16AEE
:1023100020F440600843C5F888002088800507D570
:10232000D5F88800E16B20F440200843C5F8880008
:102330002088400507D5D5F88800216C20F440108E
:102340000843C5F888002078400607D5D5F88800EE
:10235000216B20F440500843C5F88800207800061F
:1023600007D5D5F88800616B20F440400843C5F8D4
:1023700088002088C00507D5D5F88800A16B20F417
:1023800040300843C5F8880020684FF0006700031C
:102390004FF0806850D5D5F88800A16C20F04060DF
:1023A0000843C5F88800A06CB84200E005E03BD1C6
:1023B000E86840F48010E8603EE0D5F8900010F442
:1023C000407014D0A16D814211D0D5F89000D5F89D
:1023D000901020F4407041F48031C5F89010D5F889
:1023E000901021F48031C5F89010C5F89000C00716
:1023F00011D0FFF709FD074641F2883907E000BF19
:10240000FFF702FDC11B494501D9032652E7D5F864
:1024100090008007F4D5D5F89000A16D20F44070AD
:102420000843C5F8900045E7404505D10121201D2E
:1024300002F01AFB00B106462068400317D5D5F814
:102440008800E16C20F040600843C5F88800E06C2B
:10245000B84204D1E86840F48010E86007E04045E5
:1024600005D10121201D02F0FFFA00B106462088A7
:10247000400411D5D5F88800216D20F04050084364
:10248000C5F88800206DB0F1805F05D10221201DC4
:1024900002F0EAFA00B106462088000406D555F895
:1024A000880F616D20F0804008432860304600F0BE
:1024B00005B80000001002400070004018BCBDE8E4
:1024C000E08F00002DE9F0470F4605006BD0494E24
:1024D000306800F00700B84209D2306820F00700E9
:1024E00038433060306800F00700B8425BD128788C
:1024F000414C80070AD5A868A16801F0F001884224
:1025000004D9A16821F0F0010143A1602878C00737
:102510002CD06868032811D0022812D0216898B105
:10252000490500293FDAA16821F003010143A160B8
:10253000FFF76AFC804641F2883910E02168890182
:10254000EFE721688903ECE78907EAE7FFF75CFC1E
:10255000A0EB0801494502D90320BDE8F087A06837
:10256000696800F00C00B0EB810FEFD1287880078C
:102570000AD5A868A16801F0F001884204D2A168D8
:1025800021F0F0010143A160306800F00700B8427B
:102590000BD9306820F0070038433060306800F015
:1025A0000700B84201D00120D7E72878400705D5B9
:1025B000A068E96820F4E0600843A060287800077C
:1025C00006D5A068296920F4605040EAC100A060E7
:1025D00000F05EF8A168094AC1F30311515C01F0F3
:1025E0001F01C8400649086006480068BDE8F0477A
:1025F000FFF718BD00200240001002407487000859
:10260000740000204C0000200F2202600C4A9368E6
:1026100003F003034360936803F0F003836093685F
:1026200003F4E063C36092684FF4E06303EAD2020C
:1026300002610448006800F007000860704700006D
:1026400000100240002002400548064900688968E1
:10265000054AC1F30221515C01F01F01C8407047D7
:102660007400002000100240B487000805480649A5
:1026700000688968054AC1F3C221515C01F01F015D
:10268000C84070477400002000100240B487000862
:1026900070B52549002318468A68CC6812F00C02F0
:1026A00004F00306214C4FEA640509D00C2A05D03A
:1026B000042A32D0082A00D1284670BD012E10D13C
:1026C0000B681B0704D4D1F89430C3F3032302E052
:1026D0000B68C3F30313164E56F82330DAB10C2AF5
:1026E000EBD1C86800F00300022818D0032818D0E6
:1026F0001846CA68CB68C2F30212C3F306234343E9
:10270000521CB3FBF2F2C868C0F34160401C4000A9
:10271000B2FBF0F070BD184670BD204670BD20467B
:10272000E7E72846E5E70000001002400024F40037
:10273000848700082DE9F84304006FD0FA4DA8689B
:1027400000F00C06E86800F003072078C00664D5A6
:1027500076B10C2E01D1012F0AD0A069002828687B
:102760007AD040F001002860FFF74EFB80465DE024
:102770002868800702D5A0690028DED0216A286871
:10278000000703D5286800F0F00004E0D5F89400B5
:10279000F02202EA1010814216D9084602F0FAF936
:1027A00000283BD1286840F0080028602868216A8A
:1027B00020F0F000084328606868E16920F47F4059
:1027C00040EA0120686016E0286840F008002860B0
:1027D0002868216A20F0F000084328606868E169F1
:1027E00020F47F4040EA0120686026B9206A02F0A8
:1027F000D1F90028D5D1FFF74BFFA968CB4AC1F327
:102800000311515C01F01F01C840C9490860C94863
:102810000068FFF707FC00287ED12EE0CAE000BF69
:10282000FFF7F2FAA0EB0800022876D828688007A4
:10283000F6D5286840F0080028602868216A20F052
:10284000F000084328606868E16920F47F4040EAAE
:102850000120686011E0FFE720F001002860FFF729
:10286000D3FA804606E000BFFFF7CEFAA0EB0800DF
:102870000228DAD828688007F6D42078C00740D02C
:10288000082E18D00C2E01D1032F14D06068B0F59B
:10289000803F17D0B0F5A02F286817D020F48030E3
:1028A0002860286820F4802028606068E0B1FFF785
:1028B000ABFA804614E02868800322D560680028BF
:1028C00078D01EE0286840F48030EDE740F48020A6
:1028D0002860F7E7FFF798FAA0EB08006428A4D86F
:1028E00028688003F6D50CE0FFF78EFA804605E0F5
:1028F000FFF78AFAA0EB0800642896D828688003BE
:10290000F6D4207880073BD5042E11D00C2E01D1AF
:10291000022F0DD0E06801E0AAE1FFE0002828685E
:102920001ED040F480702860FFF76EFA07460CE076
:10293000286840050CD5E0680028C1D008E000BF39
:10294000FFF762FAC01B022893D828684005F7D524
:102950006868217C20F0F85040EA016068600FE070
:1029600020F480702860FFF74FFA074605E000BFAB
:10297000FFF74AFAC01B0228B1D828684005F7D4EF
:102980002078000729D560690028D5F8940012D076
:1029900040F00100C5F89400FFF736FA074604E05E
:1029A000FFF732FAC01B022899D8D5F894008007A7
:1029B000F6D512E02BE120F00100C5F89400FFF7F6
:1029C00023FA074605E000BFFFF71EFAC01B0228E6
:1029D00085D8D5F894008007F6D42078400766D5CE
:1029E000A86D0027C00008D4A86D40F08050A865ED
:1029F000A86D012700F0805000904F480168C9057C
:102A000012D40168814641F480710160FFF7FCF93E
:102A1000804605E0FFF7F8F9A0EB080002287DD812
:102A2000D9F80000C005F5D5A068012816D0052802
:102A3000D5F8900017D020F00100C5F89000D5F827
:102A4000900020F0040000BFC5F89000A06841F29B
:102A50008839C0B1FFF7D8F980460FE0D5F890006B
:102A600040F00100F0E740F00400C5F89000F5E701
:102A7000FFF7CAF9A0EB080149454FD8D5F89000F7
:102A80008007F5D50EE0FFF7BFF9804606E000BFEE
:102A9000FFF7BAF9A0EB080149453FD8D5F89000F7
:102AA0008007F5D41FB1A86D20F08050A86520786C
:102AB000800628D5606A0028D5F8980012D040F02A
:102AC0000100C5F89800FFF79FF9074605E000BF31
:102AD000FFF79AF9C01B022820D8D5F89800800784
:102AE000F6D510E020F00100C5F89800FFF78CF94A
:102AF000074604E0FFF788F9C01B02280ED8D5F876
:102B000098008007F6D4A06AF0B3022816D00C2EE5
:102B10007DD0286820F08070286000E0A7E0FFF7F3
:102B200073F90446A6E00000001002407487000814
:102B3000740000204C00002000700040E868E26A49
:102B400000F00301914228D1216B00F070020901CD
:102B50001039914221D1626B00F4FE41B1EB022F9A
:102B60001BD194F8382000F07841B1EBC26F14D13A
:102B7000A18F00F4C00249084905A1F50011914256
:102B80000BD194F8401000E06AE04908490600F0D3
:102B9000C060A1F1007181424BD00C2E73D0286827
:102BA000400170D4286820F080702860FFF72CF96D
:102BB000064604E0FFF728F9801B022857D828684A
:102BC0008001F7D4F4E90B016FF00F0202EB011161
:102BD0000843218A5204490802EB4151A26841EAA4
:102BE00002210843217D4FF07E42490802EB4161FA
:102BF0000843217B40EAC160E968244A1140084348
:102C0000E860286840F080702860E86800E03AE0FA
:102C100040F08070E860FFF7F7F8044605E000BF79
:102C2000FFF7F2F8001B022821D828688001F7D5A9
:102C300027E02868800124D4286840F0807028604C
:102C4000E86840F08070E860FFF7DEF8044604E0D2
:102C5000FFF7DAF8001B022809D828688001F7D5A9
:102C60000FE000BFFFF7D0F8001B022802D90320B5
:102C7000BDE8F88328688001F4D4E8680449084076
:102C8000E8600020F4E70120F2E700008C809D015D
:102C9000FCFFEEFE7047704770470000F0B590F8FB
:102CA0003C20012A29D0012480F83C40022280F8EF
:102CB0003D2003685A689D68114EB34203D122F447
:102CC00070074A683A4322F070070A683A435A602C
:102CD0000268B24205D0B2F1804F02D0094B9A424D
:102CE00004D1896825F080031943916080F83D4044
:102CF000002180F83C100846F0BD0220F0BD000025
:102D0000002C01400040014010B5040003D094F8AD
:102D10003D0010B107E0012010BD002084F83C0008
:102D2000204600F023F8022084F83D00211D206891
:102D300002F0E6F9012084F8480084F83E0084F8A7
:102D40003F0084F8400084F8410084F8420084F891
:102D5000430084F8440084F8450084F8460084F871
:102D6000470084F83D00002010BD00002DE9F04F21
:102D700087B0064614216846FDF7E1FA454A3168F6
:102D80004548914263D1016E41F400610166016ED4
:102D900001F400610591C16C41F00101C164C06C96
:102DA0004FF4807B00F00100CDF800B005900220C8
:102DB0000025CDE901050120CDE903505F466946B4
:102DC0004FF09040FEF730FF354C34484FF0070885
:102DD0002060C4E901854FF0800AE560C4E904A7DA
:102DE00007154FF02009A761C4E907952046FEF7B3
:102DF000FDFC08B1FDF7E4FE7462A662284C27488A
:102E0000483414302060C4E9018504F10C01A76145
:102E100081E8200CC4E907952046FEF7E7FC08B1DD
:102E2000FDF7CEFEB462002205211A20A662FFF74C
:102E30007DF91A20FFF76DF9002205211B20FFF70D
:102E400075F91B20FFF765F907B000F02FB8B1F155
:102E5000804F0BD0134A914210D1816D41F0200177
:102E60008165806D00F020000590EDE7816D41F0F7
:102E700001018165806D00F00100F5E70A4A914289
:102E8000E2D1016E41F480310166006E00F48030C1
:102E9000EAE70000002C0140001002401C00024044
:102EA000040F0020001400400040014030BCBDE889
:102EB000C08F000090F83D10012901D0012070471B
:102EC000022180F83D100168CA6842F00102CA6020
:102ED00000680B49884205D0B0F1804F02D0094903
:102EE000884207D18168084A1140062906D0B1F509
:102EF000803F03D0016841F001010160002070476C
:102F0000002C0140004001400700010070B504465C
:102F100090F83C000025012817D0012684F83C6079
:102F2000022084F83D00226890682F4B184020F45E
:102F30007F4090600868502838D00DDC20284FD0A2
:102F400005DC90B3102811D14AE0022070BD302872
:102F500046D040280AD13BE060282FD070280DD001
:102F6000B0F5805F03D0B0F5005F12D0012584F882
:102F70003D60002084F83C00284670BDCB68D1E954
:102F80000121206802F07CF92068816841F0770116
:102F900009E0CB68D1E90121206802F071F92068CD
:102FA000816841F480418160E1E719E0CA684968BD
:102FB000206802F0FDFA5021206806E0CA684968DE
:102FC000206802F02FFB6021206802F063F9CEE751
:102FD000CA684968206802F0EBFA40212068F4E7EB
:102FE000226801461046F0E788FFFEFF70477047F1
:102FF00070472DE9F041054690F83C0000260C464C
:10300000012810D0012085F83C0072B1042A1CD0A0
:10301000082A2CD00C2A50D00126002085F83C002C
:103020003046BDE8F0810220FBE7D4E90012E368F6
:10303000286802F0CFFA2868816921F00C018161CB
:1030400028688169A26811430FE0D4E90012E3689F
:10305000286802F0F9FA2868816921F440618161E9
:1030600028688169A26841EA02218161D5E7286860
:10307000D4E9002C277B016A21F480710162C169C7
:10308000036A21F0030141EA0C0121F0F00C390739
:103090004FF420674CEA116123F4206307EA02220F
:1030A0001A43C16102622868C16921F00C01C16143
:1030B0002868C169A268114328E02868D4E900277C
:1030C000E168036A23F480530362D0F81CC0036AEA
:1030D0002CF4407C4CEA07274FF6FF7C27F470471E
:1030E0000CEA013139434FF4204723F4204307EA27
:1030F00002321A43C16102622868C16921F4406149
:10310000C1612868C169A26841EA0221C16184E7FE
:1031100010B5040003D094F83D0010B107E0012081
:1031200010BD002084F83C00204600F022F8022068
:1031300084F83D00211D206801F0E2FF012084F8A1
:10314000480084F83E0084F83F0084F8400084F88A
:10315000410084F8420084F8430084F8440084F875
:10316000450084F8460084F8470084F83D000020BC
:1031700010BD70472DE9F0411F4690460D000446F2
:103180004FF0000613D0042D16D0082D19D00C2DA9
:103190001CD0102D1DD094F8430000BF94F84710A8
:1031A000022819D0022917D0012818D0B4E094F8C9
:1031B0003E0094F84410F3E794F83F0094F845106B
:1031C000EEE794F8400094F84610E9E794F84100DF
:1031D000E4E794F84200E1E70220BDE8F08101292C
:1031E00078D1B8F1000F75D0002F73D002209DB3B5
:1031F000042D37D0082D3AD00C2D3DD0102D3FD0C6
:1032000084F8430084F8470001222946206801F031
:10321000ADFF45484549464A8DB3042D46D0082D9B
:1032200059D00C2D6AD0012642492068884205D029
:10323000B0F1804F02D04049884207D181683F4AAF
:103240001140062906D0B1F5803F03D0016841F056
:10325000010101603046C0E7FFE784F83E0084F8D2
:103260004400D1E784F83F0084F84500CCE784F8B7
:10327000400084F84600C7E784F84100C2E702E056
:1032800084F84200BEE7636AD862606A3B46016325
:10329000606A4263216842463431606AFEF706FB89
:1032A000C0B92068C16841F4007111E0A36AD86216
:1032B000A06A3B460163A06A4263216842463831F6
:1032C000A06AFEF7F3FA28B92068C16841F480616A
:1032D000C160A9E720E0E36AD862E06A3B46016387
:1032E000E06A4263216842463C31E06AFEF7DEFA5A
:1032F00090B92068C16841F40061E9E7236BD862A6
:10330000206B3B460163206B42632168424640319B
:10331000206BFEF7CBFA08B101205EE72068C16898
:1033200041F48051D4E7000087510008F5510008AE
:103330002D520008002C0140004001400700010010
:1033400070B50446006801694FF00005C94389075C
:1033500015D4C168C943890711D4E91E0161012050
:103360002077206880698007204602D0FFF73FFE63
:1033700004E000F0CFF8204600F091F925772068AE
:103380000169C943490717D4C168C943490713D420
:103390006FF004010161022020772068806910F439
:1033A000407F204602D0FFF722FE04E000F0B2F892
:1033B000204600F074F9257720680169C9430907A0
:1033C00016D4C168C943090712D46FF0080101611E
:1033D000042020772068C0698007204602D0FFF7CC
:1033E00006FE04E000F096F8204600F058F9257734
:1033F00020680169C943C90617D4C168C943C90611
:1034000013D46FF010010161082020772068C06993
:1034100010F4407F204602D0FFF7E9FD04E000F001
:1034200079F8204600F03BF9257720680169C94307
:10343000C90708D1C168C943C90704D1891E016100
:10344000204600F095F920680169C943090609D4AE
:10345000C168C943090605D46FF0800101612046A7
:10346000FFF719FC20680169C943C90509D4C1687F
:10347000C943090605D46FF4807101612046FFF746
:1034800009FC20680169C943490609D4C168C943D8
:10349000490605D46FF040010161204600F09DF916
:1034A00020680169C94389060BD4C168C9438906EC
:1034B00007D46FF0200101612046BDE87040FFF79E
:1034C000EBBB70BD10B586B0044614216846FCF70E
:1034D00036FF2068B0F1804F16D10C48C16C41F026
:1034E0000201C164C06C002100F0020005904FF49D
:1034F000406000900220CDE901010390012004907A
:1035000069460348FEF790FB06B010BD001002406C
:1035100000040048704770B5044690F83C0000264F
:103520000D4601280BD0012084F83C000C2A4AD01B
:1035300007DC82B1042A20D0082A06D131E002201B
:1035400070BD102A53D0142A63D00126002084F8BD
:103550003C00304670BD206801F0A4FE20688169FF
:1035600041F0080181612068816921F004018161D5
:10357000206881692A69114311E0206801F0CEFEBC
:103580002068816941F4006181612068816921F4CA
:1035900080618161206881692A6941EA0221816133
:1035A000D4E7206801F0F6FE2068C16941F0080107
:1035B000C1612068C16921F00401C1612068C1694D
:1035C0002A69114311E0206801F01EFF2068C169DB
:1035D00041F40061C1612068C16921F48061C16169
:1035E0002068C1692A6941EA0221C161AEE7206809
:1035F00001F03AFF2068416D41F008014165206803
:10360000416D21F0040141652068416D2A69114333
:1036100011E0206801F056FF2068416D41F400611F
:1036200041652068416D21F4806141652068416DEC
:103630002A6941EA0221416588E710B5040003D0F8
:1036400094F83D0010B107E0012010BD002084F87F
:103650003C00204600F022F8022084F83D00211DA5
:10366000206801F04DFD012084F8480084F83E00F8
:1036700084F83F0084F8400084F8410084F8420058
:1036800084F8430084F8440084F8450084F8460038
:1036900084F8470084F83D00002010BD7047704753
:1036A00010B50446022269B1042912D0082917D0A6
:1036B0000C291CD0102921D094F84300012824D0D3
:1036C000012010BD94F83E000128F9D184F83E2075
:1036D0001DE094F83F000128F2D184F83F2016E065
:1036E00094F840000128EBD184F840200FE094F8D2
:1036F00041000128E4D184F8412008E094F8420018
:103700000128DDD184F8422001E084F84320012221
:10371000206801F02BFD12492068124A884204D02B
:10372000904202D0104B984203D1436C43F40043C3
:1037300043642068884204D0B0F1804F01D09042A9
:1037400007D18168094A1140062906D0B1F5803FAA
:1037500003D0016841F001010160002010BD0000AC
:10376000002C0140004001400044014007000100DE
:1037700000680349884201D1FEF73CBC7047000055
:103780000010004070B5044690F83C00012812D0AB
:10379000012584F83C50022084F83D00204601F0C9
:1037A000BFFE01004FF0000007D084F83D5084F8C0
:1037B0003C00012070BD022070BD2168CA6822F063
:1037C0004002CA602168CA6822F48042CA6084F854
:1037D0003D5084F83C00002070BD70477047704732
:1037E00070B50446806FE66F216889684FF0100558
:1037F000090618D5212816D12068083050E8001F86
:1038000021F0800140E80012002AF5D1E06E38B1C5
:10381000FDF7F2FE20B1E06EFDF788FF202821D0F1
:10382000204602F087F820688068400618D5222ECE
:1038300016D12068083050E8001F21F0400140E810
:103840000012002AF5D1206F38B1FDF7D5FE20B166
:10385000206FFDF76BFF202804D0204602F045F8CA
:10386000002070BDC4F88050032070BD70B5040006
:1038700019D02420A0672068016821F001010160AF
:103880002068002505602068456020688560204626
:1038900000F08AF9C4F88050A567E56744F8605FD6
:1038A0000020257570BD012070BD70472DE9F041E5
:1038B00002680446D0691168936840F60F052842F3
:1038C0004FF0000505D186067ED58E067CD5616E4B
:1038D0001BE1994F03F001060F40374374D0C7072F
:1038E00009D0CF0507D501271762D4F8802042F010
:1038F0000102C4F8802082070AD5DA0708D02768B9
:1039000002223A62D4F8802042F00402C4F88020F7
:1039100042070AD5DA0708D0236804221A62D4F8CD
:10392000802042F00202C4F8802002070CD501F08A
:103930002002324308D0236808221A62D4F880207B
:1039400042F00802C4F8802002050BD54A0109D5CF
:1039500023684FF400621A62D4F8802042F02002FB
:10396000C4F88020D4F88020002A35D0800605D500
:10397000880603D5616E09B120468847D4F88000D7
:1039800021688968490602D410F0280F26D0204605
:1039900001F0ABFF2068806840061AD52068083027
:1039A00050E8001F21F0400140E80012002AF5D144
:1039B000206F70B161498163206FFDF742FE0028DE
:1039C0000AD0206F816B01E00EE02046BDE8F04197
:1039D00008472046FFF769FFBDE8F0812046FFF762
:1039E00064FFC4F88050F7E7276E2026012F7BD1B3
:1039F000C70679D5CF0677D5102010622068806879
:103A0000400641D5216F086840680004000CE3D0EF
:103A1000B4F858208242DFD9A4F85A000868006838
:103A200080062AD4206850E8001F21F4807140E805
:103A30000012002AF6D12068083050E8001F21F05B
:103A4000010140E80012002AF5D12068083050E852
:103A5000001F21F0400140E80012002AF5D1E6677E
:103A60002566216851E8000F20F0100041E80002AF
:103A7000002AF6D1206FFDF7BFFDB4F85800B4F866
:103A80005A10401A81B22AE0B4F85800B4F85A101B
:103A9000401A81B2B4F85A0000289DD000299BD06A
:103AA000226852E8000F20F4907042E80003002BD7
:103AB000F6D12068083050E8002F22F0010240E8DB
:103AC0000023002BF5D1E66725666566226852E87B
:103AD000000F20F0100042E80003002BF6D1204632
:103AE000FFF77CFE78E7FFE7C70209D55B0207D541
:103AF0004FF4801010622046BDE8F041FFF76FBE22
:103B0000020606D50A0604D5A16E00297FF45DAF32
:103B100062E74006E6D54806E4D52046026852E84A
:103B2000001F21F0400142E80013002BF6D1866708
:103B3000856600F01FFA4FE720010004A357000834
:103B400010B5040002D0A06F10B107E0012010BD35
:103B5000002084F87400204600F058F82420A06764
:103B60002068016821F001010160204601F0EEFEAD
:103B70000128ECD0606A10B1204601F080FD206879
:103B8000416821F4904141602068816821F02A0158
:103B900081602068016841F0010101602046BDE8B4
:103BA000104001F0D0BD000010B50446144B016870
:103BB00014484FF09042994213D1016E21F4804194
:103BC00001664FF4C0611046FDF78CFF206FFDF7D2
:103BD0005FFDE06EFDF75CFDBDE810402520FEF7BF
:103BE00087BA094B99420AD1816D21F40031816570
:103BF000BDE8104048F204011046FDF773BF10BD48
:103C00000038014000100240004400402DE9F04718
:103C10009EB00746142117A8FCF791FB5C2168466B
:103C2000FCF78DFB4D4938684D4D002402264FF0BE
:103C300003084FF007094FF0904A88425AD10120FB
:103C4000009008946846FEF7DFFA08B1FCF7B8FF69
:103C5000286E40F480402866286E00F480401C9056
:103C6000E86C40F00100E864E86C19AA00F001007B
:103C70001C904FF4C060CDE9170682E8100317A925
:103C80005046FDF7D1FF384D36484FF08008286088
:103C9000C5E90164C5E903486C61AC61EC61284683
:103CA0002C62FDF7A3FD08B1FCF78AFF3D67AF6208
:103CB0002D4D2C4848351438E5E802061020A5E8BB
:103CC0001101294845F814494830AC61EC612C6277
:103CD000FDF78CFD08B1FCF773FFFD66002205219E
:103CE0002520AF62FEF722FA2520FEF712FA1EB059
:103CF000BDE8F0871D498842F9D1684600960994CD
:103D0000FEF782FA08B1FCF75BFFA86D40F40030C3
:103D1000A865A86D00F400301C90E86C40F001002C
:103D2000E864E86C19AA00F001001C900420CDE9B9
:103D30001706454682E8300217A957465046FDF758
:103D400073FFCDE919454FF400401B95CDE91706E7
:103D500017A93846FDF768FFC9E7000000380140A1
:103D600000100240580002409C1000200044004017
:103D700030B4C36F202B20D1E1B1DAB190F87430A8
:103D8000012B1AD0012380F87430002303660C4CF9
:103D90000368A3420BD05B681B0208D5046854E893
:103DA000003F43F0806344E80035002DF6D130BC7D
:103DB00001F0CCBE012030BC70470220FBE70000C0
:103DC0000080004010B5006810499CB088421AD1AC
:103DD00000201A9040220E496846FCF797FA0D4CD5
:103DE00000231AAA6946206804F0C8F801280AD0FE
:103DF0001AAA0AA9206804F0BDF900231AAA694684
:103E0000206804F0BBF81CB010BD00000038014071
:103E10002C11002040000020704700002DE9F843DD
:103E20000446806F1F4616460D4620284FD1CDB15F
:103E3000C6B194F87400012849D0012084F87400B8
:103E40004FF00008C4F880802120A067FDF7DCFF58
:103E5000A4F850608146A4F85260A068B0F5805F75
:103E600003D004E00120BDE8F883206928B12E4684
:103E70005FF0000584F8748010E00026FAE78021E6
:103E8000204601F0B5FEB8B9C6B116F8010B21689D
:103E90000885B4F85200401EA4F85200B4F852004D
:103EA0004B464FF0000200970028E8D14FF0400148
:103EB000204601F09DFE30B10320D4E735F8020B17
:103EC000C0F30800E3E72020A0670020CBE7022032
:103ED000C9E7000070B50446806F202841D169B35E
:103EE00062B394F8740001283BD0012084F8740078
:103EF000E164A4F85020A4F852200025C4F88050B2
:103F00002120A067E06ED8B11749C162E16E174861
:103F100013460863E16E16484863E06E85632668C1
:103F2000E16C06F12802E06EFDF7C0FC40B1102004
:103F3000C4F8800004F8745F20206060012070BD28
:103F400021684020086284F874502068083050E8E6
:103F5000001F41F0800140E80012002AF5D1002046
:103F600070BD022070BD00009F580008E158000895
:103F7000B757000800680449884204D10022202174
:103F80000248FDF73CBF704700380140000400487C
:103F90007047FEE7134D144E0024287850B10128D5
:103FA0000AD002280AD003280AD000203178032939
:103FB00008D008E00220F9E70320F7E70420F5E73E
:103FC0000520F3E70620A04202D0044601F0B0FE2F
:103FD000064800F00FF8064800F00CF80A2002F03E
:103FE000C1FCDAE70000002024010020C40000200A
:103FF000B000002010B50446807A002832D0E28854
:10400000002A2FD020890A3081B22181A37C002090
:1040100053B1E289914225D320812073A074E074CA
:10402000A188002220680BE091421BD32081E07C14
:1040300050B10020E0740028A188206806D0012239
:10404000BDE81040FDF7DBBE0120F3E70022FDF7DD
:10405000D6FE207B401CC0B22073E17A884201D397
:104060000120A07410BD00EB8100006E00F0F8404C
:1040700070478068C0F3C00070478068C0F380005C
:104080007047C06810F4406F01D0002070470120D5
:104090007047042303EAD15310B518444369C1F3B0
:1040A000045107248C40A3438A401343436110BD4D
:1040B00000EB8100016E21F0004111430166704761
:1040C00010B586B018216846FCF739F931483049F7
:1040D00000F10C0301600021416001220424816091
:1040E00083E81600017642760523C36180F820102C
:1040F0008162C16280F830201203426380F8381078
:10410000FDF7D4F808B1FCF75BFD234800900620CA
:104110000190072002907F2003900320CDE9040442
:1041200069461C48FCF7C6FE08B1FCF749FD1B4870
:1041300000900C20019069461648FCF7BBFE08B1C0
:10414000FCF73EFD16480090122001906946114888
:10415000FCF7B0FE08B1FCF733FD124800901820C0
:10416000019069460B48FCF7A5FE08B1FCF728FD55
:104170000D4800904FF48070019069460548FCF7A7
:1041800099FE002801D0FCF71BFD06B010BD000011
:1041900000000450D40C00200002B0250004002AC6
:1041A0000008302E0010603200002143194808B585
:1041B000816C41F001018164806C002200F00100FB
:1041C000009005210B20FDF7B1FF0B20FDF7A1FFAB
:1041D000002205210C20FDF7A9FF0C20FDF799FF17
:1041E000002205210D20FDF7A1FF0D20FDF791FF15
:1041F000002205210E20FDF799FF0E20FDF789FF13
:10420000002205210F20FDF791FFBDE808400F2097
:10421000FDF77FBF0010024010B517A001F050FE5F
:10422000194A2821402002F0D9FB184C164A0021D7
:104230002064B43A164802F0FDFB134AE062903A5B
:104240000021144802F0F6FB0F4A20636C3A00216B
:10425000114802F0EFFB0C4A6063483A00210F4816
:1042600002F0E8FB084AA063243A00210C4802F05F
:10427000E1FBE06310BD0000415049325F454C4511
:1042800020303631320D0A005C8700080000002023
:10429000953F0008DD4D0008114C00085D4E0008F8
:1042A000514600082DE9F04186B014216846FCF71C
:1042B00046F82348C16C41F00101C164C16C01F0B2
:1042C00001010591C16C41F00201C164C06C1D4F38
:1042D00000F002000590012241F204013846FDF78A
:1042E0008EFD4FF4C0564FF09048002231464046B4
:1042F000FDF785FD0022E0213846FDF780FDE42032
:10430000009001250024CDE9015469463846039404
:10431000FDF78AFC2803CDE900050320CDE9024022
:1043200069463846FDF780FC0096CDE901546946A0
:1043300040460394FDF778FC06B0BDE8F08100002C
:104340000010024000040048134810B511490160F4
:104350001249416000210122C0E90212016141615C
:104360008161C1610162FDF7A9FD08B1FCF728FC7C
:1043700000210948FDF74EFD08B1FCF721FC0021A2
:104380000548FDF772FD002803D0BDE81040FCF79A
:1043900017BC10BD00580040800D0020694EA530AC
:1043A00010B588B000241848009401940294039436
:1043B000049405941349069401604F21C0E9011447
:1043C0004FF6FF71C0E9031444618461FEF79CFC61
:1043D00008B1FCF7F5FB4FF48050009069460A489D
:1043E000FEF794FD08B1FCF7EBFB049404A9064822
:1043F0000694FEF753FC002801D0FCF7E1FB08B05F
:1044000010BD000000400140B80E002010B590B073
:1044100000240C940D940E94142104A80F94FBF71F
:104420008EFF2E480A940B940994009401940294F0
:104430002949039401604F21C0E901144FF6FF712F
:10444000C0E903148021C0E90541FEF75DFC08B115
:10445000FCF7B6FB4FF480500C900CA91F48FEF7F8
:1044600055FD08B1FCF7ACFB1C48FEF751FE08B146
:10447000FCF7A6FB042004905020CDE9050404A914
:1044800016480894FFF77EF908B1FCF799FB0994E8
:104490000A9409A911480B94FEF700FC08B1FCF737
:1044A0008FFB0120CDE900400294002269460B48B1
:1044B0000394FEF79EFD08B1FCF782FB02200090FA
:1044C0000190042269460548FEF793FD002801D0BB
:1044D000FCF776FB10B010BD002C0140D40D00207D
:1044E00010B58EB000240794089409940A940B9494
:1044F0000C941C2168460D94FBF721FF22484FF0D5
:10450000804101602721C0E9011440F2E731C0E990
:1045100003148461FEF7F8FB08B1FCF751FB4FF47C
:104520008050079007A91848FEF7F0FC08B1FCF787
:1045300047FB1548FFF781F808B1FCF741FB0B94E6
:104540000BA911480D94FEF7A9FB08B1FCF738FB45
:10455000602000904FF4FA70CDE90104082269460A
:1045600009480494FEF7D7FF08B1FCF729FB0C2299
:1045700069460548FEF7CFFF08B1FCF721FB02486A
:10458000FEF7A0FF0EB010BD200E00203EB50024A7
:104590000F48009401940D49029401604F21C0E935
:1045A00001144FF6FF718461C160FEF7ADFB08B1E5
:1045B000FCF706FB0094694605480294FEF76EFB83
:1045C000002801D0FCF7FCFA3EBD000000140040BA
:1045D0006C0E00200D4810B50B4901604FF41651C8
:1045E0004160002181600C22C160C0E90412816138
:1045F000C16101624162FFF7A3FA002803D0BDE860
:104600001040FCF7DDBA10BD00380140940F0020C7
:104610000D4810B50B4901604FF47A31416000211B
:1046200081600C22C160C0E904128161C161016234
:104630004162FFF785FA002803D0BDE81040FCF77F
:10464000BFBA10BD0044004018100020FEE7000073
:1046500008213C48FFF724F80C213A48FFF720F8DE
:10466000002600F0D1F8DFF8E090DFF8E0B0384F36
:10467000DFF8D080002400BF99F80000A8B33549C6
:10468000F868884210DD40F2DC50864202D20A36D9
:10469000B6B20AE003218BF80010D8F80010CC6302
:1046A000D8F80000046400E00026DFF8ACA0D7EDE5
:1046B000040A50469AED020A00F067F8BDEEC00AFF
:1046C00040F2BA2110EE100A05B205F25D108842E0
:1046D0000DD89AED020AB5EEC00AF1EE10FA06D036
:1046E000002D03DD4FF4FA7501E018E01B4D9BF837
:1046F0000000DA46012802D1A8B200F031F89AF899
:104700000000022802D1A8B200F034F89AF80000A4
:1047100028B9D8F80010CC63D8F8000004643878C1
:1047200040B1D8F800100C64022806D0032804D049
:10473000012802D0D8F80000C4630A2002F012F960
:104740009AE70000200E002018010020240100201C
:1047500000000020295C0F3D841200200CFEFFFFAA
:1047600003490A68D06309680020086470470000A4
:10477000200E0020034900220B68DA6309680864F0
:1047800070470000200E0020FEE730EE600AB0EE19
:10479000002A80ED030AD0ED040AD0ED071A30EEAE
:1047A000601A21EE211AD0ED081A01EE801AD0ED20
:1047B000061A70EE211A40EEC21A90ED092A02EE96
:1047C000211AD0ED0A1A31EE211A80ED0A1AC0ED35
:1047D000060A80ED040A90ED0B0AB4EEC01AF1EE61
:1047E00010FA01DD80ED0A0AD0ED0A0AB1EE400AA6
:1047F000F4EEC00AF1EE10FA02D3B0EE600A704790
:1048000080ED0A0A7047000015489FED140ADFED9D
:10481000150A80ED000A80ED010AC0ED020A80ED64
:10482000030A80ED040A80ED050A9FED0F0A80ED72
:10483000070A9FED0E0A80ED080A9FED0D0A80ED34
:10484000090A9FED0C0A80ED0B0A9FED0B0A80ED23
:104850000C0AB1EE040A80ED0D0A7047000000005A
:1048600084120020000048436666A63F3333333F7E
:10487000CDCC4C3E00007A4400007AC470B52DEDDA
:10488000048BFDF7C1FA05465448406A0068406849
:104890000A21C0F10A00B0FBF1F201FB12005049FD
:1048A000504A51F8201052F8200000286FD000EE36
:1048B000101AF8EE400A00EE100AB8EE401A80EE28
:1048C000810ADFED490A20EE200A9FED481A484C84
:1048D00020EE018A94ED060A9FED461A00EE018A49
:1048E00084ED028A206A281A01EE100AB8EE411AF5
:1048F000DFED411A4149C1EE218A18EE900A884243
:1049000069DD38EE400A3E49C4ED058A10EE100A12
:10491000884202DD30EE600A06E010EE100A3949E6
:10492000884201D930EE200AB2EE049A20EE090A3C
:1049300001F0E6FAC0EE090A3349B0EEE00A10EEE3
:10494000100A884202DAC0EEA82A01E0D4ED092A52
:1049500094ED090A2D4972EEC00AF0EEE00A10EE5D
:10496000900A884201DDF0EE402A294800780128AB
:1049700002D002280CD015E0F5EEC02AF1EE10FAB4
:1049800002D2D4ED0A2A0DE0C4ED0A2A0AE022E0A0
:10499000F5EEC02AF1EE10FA02DDD4ED0B2A01E0AB
:1049A000C4ED0B2A18EE100A1A4908441A49884225
:1049B00006D318EE100A194908441949884201D251
:1049C000F0EE402AB0EE620A01F008FAC4ED092ABE
:1049D000256284ED068ABDEC048B70BDD40D0020E9
:1049E0005C020020340200200000B443CDCC4C3ED9
:1049F00078000020CDCC4C3F00007A446F12833AFF
:104A000000003443000034C3000070420000C8437B
:104A100024010020FFFF8FBEFFFFEB00FFFF50BC13
:104A200032F3040000B591B028216846FBF787FCFB
:104A30000C4800226946006803F000FB012807D1FA
:104A4000684601F015FF0028684603D002F064F8BC
:104A500011B000BD01F02EFF0028F9D0684602F029
:104A6000A1F8F5E7400000202DE9F041444C05464F
:104A70008846E0680026810728680DD0E16801F0CB
:104A80000301814216D1A8B1E0686968C0F3021041
:104A9000401C88420ED120E0012804D0022805D015
:104AA000032807D108E02168890701E0216849054A
:104AB000002907DB01265FE02168890302D4216811
:104AC0004903F5E7E1686A686FF00F0321F07301AD
:104AD00003EB021211430143E160206820F0806083
:104AE0002060FDF791F9074605E000BFFDF78CF95E
:104AF000C01B022837D820680001F7D4B8F1000F96
:104B000018D0B8F1010F1DD0287D4FF07E4140082C
:104B100001EB4060A96840EA01202169194A11406F
:104B200008432061206840F080602060FDF76CF948
:104B300007461AE0A868297B000240EAC1602169A3
:104B4000114AECE7288A1149400801EB4050A96856
:104B500040EA012021690E4AE1E700BFFDF754F960
:104B6000C01B022801D9032606E020680001F5D504
:104B70002069A969084320613046BDE8F081000042
:104B800000100240FF80FFF9FF80FF070000E0FFF8
:104B9000FF809FFFF8B51C4D06460024A86DC0009D
:104BA00002D5FDF729FB0DE0A86D40F08050A86507
:104BB000A86D00F080500090FDF71EFBA96D21F05C
:104BC0008051A965B0F5007F04D0802E07D94FF041
:104BD00003040AE0802E08D9A02E01D804E001D1F8
:104BE000022402E0702E00D101240848016821F05F
:104BF000070121430160006800F00700A04201D0D6
:104C00000120F8BD0020F8BD001002400020024045
:104C10002DED048B6148FBF73DFF7F215F48FCF7DA
:104C200001F905225E495D48FCF78CFC5C4D9FED67
:104C30005D8ADFED5D8ADFF874A1DFF874915D4F66
:104C4000DFF874815D4C5E4EB0EE009A4FF0010BC0
:104C50002B88A38000EE103A6A88E280B8EE400A02
:104C6000A9882181E88820EE080A6081B5F808C08B
:104C7000A4F802C020EE280A84ED050A00EE102AEE
:104C8000B8EE400A20EE080A20EE280A84ED060A53
:104C900000EE101AB8EE400A20EE080A20EE280AAC
:104CA00084ED070A00EE100AB8EE400A20EE080A6A
:104CB00020EE280A84ED080A00EE10CAB8EE400A79
:104CC00020EE080A20EE280A10EE100A84ED090AE8
:104CD000504503DD9FED3B0A84ED090A20EE090AE9
:104CE00084ED0A0A84ED030A01F006FF01F0F0FEEC
:104CF0006069414600EB09038B420CD2A369BB42B9
:104D000009DDDFF8C4C0236A634504DDB3F17F5FCA
:104D100001DA00200EE000EB09028A420DD2A269FE
:104D2000BA420ADD226AB2F17F5F06DDB2F1804F3E
:104D300003DA5846207030802CE04FF07E539842C2
:104D40000FDAA2699A420CDD204B9A4209DA184B1D
:104D5000226ADB439A4204DDB2F1804F01DA02207D
:104D600015E01B4A1044404510D21A49A0698842F8
:104D70000CDD1949884209DA0D49206AC943884285
:104D800004DDB0F1804F01DA032000E00420207040
:104D9000A6F800B0642001F0E5FD59E7D40C00202E
:104DA000280200200000803933335340333353400E
:104DB000323333C000002040323333000000002083
:104DC0009401002000000000CDCC8C3F3333B33F72
:104DD000656666C06666663F6666A63F0A230B4A3E
:104DE00000210B48FEF7C6F9084A0A23283204219D
:104DF0000748FEF7BFF900BFFFF714FE01F05EFEA3
:104E000001F070FE052001F0ADFDF5E73402002051
:104E1000D40D002070B50E48FEF7E2FC0C4C206863
:104E2000016821F0100101600A4900204FF48075EB
:104E3000088029460848FBF782FA2A460649204698
:104E4000FEF796FF2068016841F01001016070BD17
:104E5000940F0020440000202C1100201FB52A4888
:104E6000008900F0A1F8FFF7D5FFDFF8A090DFF888
:104E7000A0A0DFF8A0B0DFF8A08000BF99ED000A85
:104E80008AED000A99ED030A8BED000AD8F80C00B0
:104E9000FBF774FA06460F46D8F81000FBF76EFAD7
:104EA00004461E480D460068FBF768FA8DE8F000DE
:104EB00041EC100B1AA053EC102B01F001F8C820A4
:104EC00001F050FD98F8000010B923A000F0F8FFA1
:104ED00098F800004446012802D123A000F0F0FF1A
:104EE0002078022802D124A000F0EAFF20780328CD
:104EF00002D125A000F0E4FF20780428BED126A02E
:104F000000F0DEFFBAE700008201002084120020DA
:104F10001C01002020010020000000208000002053
:104F20006375725F616E676C655F6465673D5B2585
:104F30002E32665D204D6F746F725F7370655B25F6
:104F40002E32665D204D6F746F725F6375725B25E4
:104F50002E33665D0D0A0000436C6F7365206F751C
:104F600074707574200D0A00436C6F736520696E50
:104F7000707574200D0A00004F70656E3120696EE7
:104F8000707574200D0A00004F70656E3220696ED6
:104F9000707574200D0A000064656661756C745F3D
:104FA00048616C6C200D0A0010B54FF416510928A9
:104FB0001AD2DFE800F0190519080B0E11141700BA
:104FC0004FF4965110E04FF496410DE04FF4164126
:104FD0000AE04FF4614107E04FF4E13104E04FF49F
:104FE000613101E04FF47A310F480E4AC0E90021E7
:104FF000002181600C22C160C0E904128161C1619D
:1050000001624162FEF732FC08B1FBF7D9FD0648A8
:10501000FEF796FD002803D0BDE81040FBF7D0BD99
:1050200010BD000000380140940F002010B54FF073
:10503000E020006903F082F9012803D0BDE81040A8
:1050400002F03EBE10BD00B597B044216846FBF7A4
:1050500076F9142111A8FBF772F94FF40070FDF7EF
:1050600097F808B172B6FEE70220C1010391102142
:10507000009004910A900121CDE90B010A210D91C4
:105080000721CDE90E1010906846FDF753FB08B1DB
:1050900072B6FEE70F2011900320129000201390AB
:1050A00014901590042111A8FDF70CFA002801D0E6
:1050B00072B6FEE717B000BD0248016841F4700106
:1050C0000160704788ED00E010B50648FEF738F93A
:1050D000002201211B20FDF729F8BDE810401B200C
:1050E000FDF717B8D40D00200148FEF729B90000DC
:1050F000D40D00200148FEF723B900002C12002037
:1051000070B50268164B4FF08046984201D0B0420D
:1051100003D122F070044A682243124C124D984287
:1051200005D0B04203D0A04201D0A84203D122F45E
:105130004076CA6832434E6922F0800232430260F0
:105140008A68C2620A688262984203D0A04201D093
:10515000A84201D1096901630121416170BD0000CC
:10516000002C0140004001400044014010B501F016
:105170001F030121046A99408C430462016A9A402A
:105180001143016210BD10B5846A0121626A824236
:1051900007D12177C06938BB84F83E1084F84410E9
:1051A00022E0A26A824208D102222277C069D8B9DD
:1051B00084F83F1084F8451016E0E26A824208D174
:1051C00004222277C06978B984F8401084F8461028
:1051D0000AE0226B824207D108222277C06918B9FF
:1051E00084F8411084F847102046FDF700FF0020A6
:1051F000207710BD10B5846A616A814201D1012017
:105200000DE0A16A814201D1022008E0E16A8142F9
:1052100001D1042003E0216B814201D108202077D5
:105220002046FDF7E5FE0020207710BD10B5846A0A
:105230000121626A824203D1217784F83E1019E08D
:10524000A26A824204D10220207784F83F1011E044
:10525000E26A824204D10420207784F8401009E0F9
:10526000226B824204D10820207784F8411001E0AB
:1052700084F83D102046FDF7B9FE0020207710BDD0
:1052800010B5846842EA032224F47F440A4322438F
:10529000826010BD826822F070020A4342F007016A
:1052A00081607047F0B5026A22F001020262056A6D
:1052B00043688269154C25F0020522400C6822F0F3
:1052C000030214438A68134E2A43114D124FA84219
:1052D00003D0B04201D0B84206D122F0080CCA680F
:1052E00042EA0C0222F00402A84203D0B04201D0EC
:1052F000B84205D14D6923F440731D438B692B439C
:1053000043608461496841630262F0BD8FFFFEFF24
:10531000002C0140004001400044014030B5026AC9
:1053200022F010020262046A42688369154D2B4024
:105330000D6823F4407343EA052524F020038C68AC
:1053400043EA0413104CA04207D1CC6823F0800339
:1053500043EA041323F0400305E00C4CA04202D0C2
:105360000B4CA04207D14C6922F4406242EA84020D
:105370008C6942EA84024260856149688163036204
:1053800030BD0000FF8FFFFE002C014000400140B7
:105390000044014030B5026A22F480720262046A5D
:1053A0004268C369144D2B400D6823F003031D436D
:1053B00024F400738C6843EA0423104CA04207D104
:1053C000CC6823F4006343EA042323F4806305E0FC
:1053D0000B4CA04202D00B4CA04207D14C6922F4E6
:1053E000405242EA04128C6942EA04124260C561EA
:1053F0004968C163036230BD8FFFFEFF002C01408E
:10540000004001400044014030B5026A22F480525D
:105410000262046A4268C3690F4D24F400542B40B1
:105420000D6823F4407343EA05238D6844EA05348C
:105430000A4DA84205D00A4DA84202D0094DA84203
:1054400004D14D6922F4804242EA85124260C36170
:1054500049680164046230BDFF8FFFFE002C0140EB
:10546000004001400044014030B5026A22F480321D
:105470000262046A4268436D0E4D2B400D681D4365
:1054800024F400330C8943EA04430B4CA04205D0BA
:105490000A4CA04202D00A4CA04204D14C6922F42A
:1054A000803242EA042242604565496881650362B0
:1054B00030BD00008FFFFEFF002C01400040014086
:1054C0000044014030B5026A22F480120262046A8C
:1054D0004268436D0E4D24F400142B400D6843EADE
:1054E00005230D8944EA05540A4DA84205D00A4D0A
:1054F000A84202D0094DA84204D14D6922F480226D
:1055000042EA8522426043654968C165046230BD54
:10551000FF8FFFFE002C014000400140004401408D
:1055200070B505680024AA6822F070034A681A431F
:105530001E4B1A400B681343AB604A6812F00F0F02
:1055400031D11211082A2ED2DFE802F02E2E2E2E93
:105550000B2127040B69D1E902210068FFF790FEB7
:1055600022E00A68052A10D00268136A156A25F03D
:105570000105156202689569096925F0F00545EA9B
:1055800001119161006803620EE0012070BD0A699B
:105590008968006800F00CF806E00A69896800680C
:1055A00000F040F800E00124204670BDF8FFFEFF47
:1055B00010B5036A046A24F001040462846924F0CB
:1055C000F00444EA021423F00A020A4384610262EE
:1055D00010BD000070B5046A24F0010404628469FF
:1055E000056A0E4EB04205D0B0F1804F02D00C4E8D
:1055F000B04203D124F00304144301E044F0010459
:105600001A0724F0F00444EA126225F00A0301F0BC
:105610000A0119438261016270BD0000002C014043
:105620000040014010B5036A23F010030362836950
:10563000046A23F4704343EA023224F0A00343EAED
:1056400001118261016210BD30B5046A24F01004BA
:1056500004628469056A24F4407444EA022222F454
:1056600070444FF6FF7202EA03322243A02425F071
:10567000A00304EA011119438261016230BD90F870
:105680002410C90706D001684A68836A22F40032F0
:105690001A434A6090F82410890706D501684A68C1
:1056A000C36A22F480321A434A6090F824104907F2
:1056B00006D501684A68036B22F480221A434A60C7
:1056C00090F82410090706D501684A68436B22F454
:1056D00000421A434A6090F82410C90606D50168B2
:1056E0008A68836B22F480521A438A6090F82410EF
:1056F000890606D501688A68C36B22F400521A43F2
:105700008A6090F82410490611D501684A68036C34
:1057100022F480121A434A60016CB1F5801F06D151
:1057200001684A68436C22F4C0021A434A6090F848
:105730002410090606D501684A68806C22F400220C
:1057400002434A607047F8B500260446C0F88060FE
:10575000FCF75AFB0546206800686FF07E4700079B
:1057600008D52B4600224FF400112046009700F088
:105770003FFA60B92068006840070AD52B4600222E
:105780004FF480012046009700F032FA08B1032060
:10579000F8BD2020A067E067266684F874600020CA
:1057A000F8BD10B5806A0021A0F85A10A0F8521078
:1057B000FEF77BF810BD70B5846AA06FE56F2168B5
:1057C00089684FF00006090606D5212804D1A4F8FF
:1057D0005260204600F0AEF820688068400606D58A
:1057E000222D04D1A4F85A60204600F07EF8D4F8A7
:1057F000800040F01000C4F880002046FEF755F805
:1058000070BD10B50146806A0968096889062DD403
:105810000021A0F85A10016851E8002F22F480728C
:1058200041E80023002BF6D10168083151E8002F30
:1058300022F0010241E80023002BF5D10168083174
:1058400051E8002F22F0400241E80023002BF5D15F
:105850002021C167016E012908D1026852E8001FAA
:1058600021F0100142E80013002BF6D1016E01294E
:1058700002D0FEF7A7FA10BDB0F85810FDF7AEFF42
:1058800010BD10B5806A016E012902D0FEF7C4FA7E
:1058900010BDB0F858104908FDF7A0FF10BD10B5B5
:1058A0000146806A09680968890616D40021A0F8B3
:1058B00052100168083151E8002F22F0800241E8BF
:1058C0000023002BF5D1026852E8001F41F040018F
:1058D00042E80013002BF6D110BDFEF74BFB10BDC4
:1058E00010B5806AFEF754FB10BD016851E8002F27
:1058F00022F4907241E80023002BF6D101680831B0
:1059000051E8002F22F0010241E80023002BF5D1DD
:10591000016E012908D1026852E8001F21F0100130
:1059200042E80013002BF6D12021C1670021016657
:1059300041667047026852E8001F21F0C00142E84A
:105940000013002BF6D12021816770472DE9F0412B
:105950000446016880682269E36910436269002592
:105960001A431043714F0A68714B1A4002430A6090
:1059700020684168E26821F4405111434160216888
:10598000A069B94201D0226A10438A6822F43062C9
:1059900002438A606749236867488B420DD1D0F87B
:1059A000880010F0030006D0012847D0022843D019
:1059B000032830D144E001212EE060498B420BD115
:1059C000D0F8880010F00C0034D0042836D0082815
:1059D00032D00C281FD133E059498B420BD1D0F87B
:1059E000880010F0300025D0102827D0202823D0A0
:1059F000302810D124E0BB420DD1D0F8880010F43B
:105A0000406017D0B0F5806F18D0B0F5006F13D09C
:105A1000B0F5406F14D010214A4A00264FF40040E0
:105A2000BB422FD171B102290FD004290FD0082910
:105A300073D10FE00021EFE70221EDE70421EBE74E
:105A40000821E9E7FCF700FE03E0104602E0FCF75E
:105A50001FFEE8B3626802EB420181425DD8B0EB01
:105A6000023F5AD8010E0302500818187141002352
:105A7000FAF718FC344AA0F5407191424DD82168DC
:105A8000C8604BE0E3694FF6EF77834228D10929DC
:105A900043D2DFE801F005080B420D4242421000FC
:105AA000FCF7D2FD06E0FCF7E1FD03E0104602E062
:105AB000FCF7EEFD60B14100606801EB5001B1FB05
:105AC000F0F0A0F11001B94227D84FF6F07100E0D4
:105AD00024E00140C0F3420001432068C1601DE0A2
:105AE00009291AD2DFE801F005080B190D19191957
:105AF0001000FCF7A9FD06E0FCF7B8FD03E0104636
:105B000002E0FCF7C5FD48B1616800EB5100B0FB55
:105B1000F1F0A0F11001B94205D9012566662846C9
:105B2000A666BDE8F08180B2A9E7000000800040D1
:105B3000F369FFEF003801400010024000440040CC
:105B4000004800400024F400FFFC0F0070B54165E0
:105B5000A0F8582000250446C0F880502220E067B5
:105B6000206FD8B11F49C162216F1F4813460863D7
:105B7000216F1E484863206F8563666D2168324639
:105B80002431206FFBF792FE40B11020C4F8800052
:105B900004F8745F2020A060012070BD84F8745068
:105BA000206940B1216851E8000F40F4807041E85D
:105BB0000002002AF6D12068083050E8001F41F0AA
:105BC000010140E80012002AF5D12068083050E8B1
:105BD000001F41F0400140E80012002AF5D10020EA
:105BE00070BD00000358000883580008B75700082C
:105BF0002DE9F0479A4617460E4604464FF0000935
:105C00004FF02008089D4AE0681C48D0FCF7FCF8DB
:105C1000A0EB0A00A8422AD84DB3206801684907C2
:105C20003DD5C069C043000539D421684FF40060F8
:105C30000862206850E8001F21F4D07140E800128B
:105C4000002AF6D12068083050E8001F21F0010139
:105C500040E80012002AF5D1C4F87880C4F87C80AE
:105C6000C4F8808084F874900320BDE8F087216830
:105C700051E8000F20F4D07041E80002002AF6D16C
:105C80002068083050E8001F21F0010140E80012B0
:105C9000002AF5D1C4F87880C4F87C80E2E7206857
:105CA000C06936EA000004D00020B842ACD0002021
:105CB000DBE70120F9E7000010B51A4C2068C16944
:105CC000C943C90614D4102101622046FDF788FD9E
:105CD0001548006840681549C0F5807080B208809A
:105CE000401EFF2802D82046FEF76CF8FFF792F816
:105CF0002068C169090705D4C169490702D4C1698F
:105D0000890709D5082101622168042008622168F9
:105D100002200862FFF77EF8BDE810400148FDF759
:105D2000C5BD0000940F00209C10002044000020FE
:105D30002DE9F0470121274C0D03642600234FF085
:105D400090494FF4FA7C4FF4FA67A4F11402072843
:105D50003ED2DFE800F0040C121920273200A372B3
:105D60009372012240211C48FCF749F829E0A172F6
:105D7000A4F806C09372BDE8F087A172A4F806C02B
:105D80009172D680D17214E0A172A4F806C091720B
:105D9000D68002200CE0A172A4F806C09172D680D1
:105DA000032005E0A172A4F806C09172D6800420F9
:105DB000D072D78113739374DDE7A172A4F806C083
:105DC000937229464846BDE8F0470122FCF717B810
:105DD000A372CFE7C40000200004004830B5334A66
:105DE0003148D16900EB8103491C83ED000A03238C
:105DF00091FBF3F403FB1411D161D0ED000A2C4A9E
:105E0000F5EEC00AF1EE10FA36D0D0ED010AF5EE4B
:105E1000C00AF1EE10FA2FD0D0ED020AF5EEC00A5A
:105E2000F1EE10FA28D08C1C94FBF3F503FB15441B
:105E300000EB8404F6EE001A94ED001A4C1C94FB5F
:105E4000F3F503FB154300EB830300EB8100D3ED77
:105E5000000A90ED000A10EE901A164881420EDA00
:105E600011EE101A81420ADD10EE101A814206DD91
:105E700031EE000A20EE210A82ED000A30BD30EE3C
:105E8000C12A0D48B0EEC22A12EE101A814207DD77
:105E900030EEC02AB0EEC22A12EE101A8142E7DCC0
:105EA000C2ED000A30BD000078120020780000200A
:105EB000100000200000A04200002042FEE7000089
:105EC0000FB4054B10B503A9044A029800F02AF953
:105ED00010BC5DF814FB0000596800082402002083
:105EE0000907090E002804DB00F1E02080F8001407
:105EF000704700F00F0000F1E02080F8141D70479B
:105F000010B52DED028BB0EE408A18EE100AFAF7AC
:105F10007DFA01EE100A18EE100AB7EE000A78EECC
:105F2000410A10F0004F4FF07F4010EE901A12D04F
:105F3000B1F13F4F24BF10EE901AB0EB410F12D2D7
:105F400010EE901AB1F17C5F1CDD10EE901AB0EBF0
:105F5000410F17D314E0B1F13F4F07D910EE901A5B
:105F6000B0EB410F02D331EE401A0BE010EE901A65
:105F7000B1F17C5F06DB10EE901AB0EB410F01D35C
:105F800031EE001A18EE100ABDEC028B11EE101A59
:105F900061F31E0000EE100A10BD02E008C8121FD7
:105FA00008C1002AFAD170477047002001E001C102
:105FB000121F002AFBD170472DE9FF5FDDE90220A7
:105FC000010DDDF838B0024318D044F61050A1F2AC
:105FD000FF3141430D140F98012820D0A5EB0B0091
:105FE000401C5FEA000A4FF00004474EDFF81C91A6
:105FF000A046504616D5CAF1000728E00F980124A4
:1060000043A2012808D0002100980F9BC0E900217D
:10601000C0E9024300F082B86FEA0B01F4E7CBF16C
:106020000000DEE7074612E0F80707D022463346B5
:1060300040464946FAF7B7FA804689462246334633
:1060400010461946FAF7AFFA04460E467F10002FA5
:10605000EAD1DDE90201BAF1000F42464B4602DA0D
:10606000FAF7A1FA01E0FAF713FB04460E46002204
:10607000284BFAF795FB03D84FF0FF30014607E0B5
:106080000022254B20463146FAF7DEF9FAF76FFB7E
:10609000102409E0002C0ADB0A220023FAF702F997
:1060A000019B30321A55641E50EA0102F2D1641C81
:1060B000019AC4F1110314440F9A012A03D001225A
:1060C00008430DD10AE0084304D000204FF0110B23
:1060D0000F9080E7A3EB0B056D1E0DE05B4504DD23
:1060E0004FF0000205F1010504E003DA4FF0000271
:1060F000A5F10105002AECD000980F99C0E9023102
:10610000C0E9004586E70000000024400000F03FA1
:10611000300000000000F0430000E03F3FBCBDE85D
:10612000C09F00002DE9FF4F95B09B46894606466B
:1061300000250FE2252877D100242746F84A0121BF
:10614000059400E0044316F8013F203B01FA03F0F8
:106150001042F7D130782A2811D06FF02F03307811
:10616000A0F13002092A16D8059A44F0020402EB85
:10617000820203EB42021044761C0590EFE759F8C7
:10618000042B0592002A03DA504244F4005405908F
:1061900044F00204761C30782E2816D116F8010F30
:1061A00044F004042A280DD06FF02F023078A0F1BB
:1061B0003003092B09D807EB870302EB4303C71809
:1061C000761CF3E759F8047B761C30786C280FD0E6
:1061D00006DC4C2817D068280DD06A2814D104E0BA
:1061E000742810D07A280FD10DE044F400140AE08E
:1061F00044F4801401E044F440147278824202D1E5
:1062000004F58014761C761C307866280BD013DCDD
:10621000582877D009DC002875D04528F6D04628C4
:10622000F4D047281AD19DE118E0632835D06428BE
:1062300079D0652812D195E1702873D008DC6728E1
:10624000F1D069286FD06E280DD06F2806D1B5E047
:1062500073282CD0752875D0782874D05A46179991
:1062600090476D1C75E1C4F30250022809D0032841
:106270000DD0D9F8001004280DD00D6009F10409E3
:1062800067E1D9F80010EA17C1E90052F6E7D9F83A
:1062900000100D80F2E70D70F0E719F8041B8DF87F
:1062A000001000208DF80100EA46012003E059F8B3
:1062B00004AB4FF0FF3061074FF0000102D40DE056
:1062C00008F101018846B9420FDA8045F8DB1AF877
:1062D00008100029F4D108E008F101018846814244
:1062E000FADB1AF808100029F6D105985B46A0EBF6
:1062F000080721463846179A00F097FA284400EB21
:10630000080507E04DE029E10DE01AF8010B5A46B7
:1063100017999047B8F10108F7D25B4621463846F5
:10632000179A13E142E00A220092C4F302524FF09E
:10633000000A022A08D059F804CB032A4FEAEC716C
:106340000AD00DE029E02AE009F1070121F0070257
:10635000F2E802C1914609E00FFA8CFC4FEAEC71B9
:10636000042A03D14FFA8CFC4FEAEC71002907DABA
:106370000A460021DCF1000C61EB02012D2202E053
:10638000220504D52B228DF80420012203E0E20728
:1063900001D02022F7E7904659E00A2102E01022BE
:1063A0000DE010214FF0000A00910BE010224FF099
:1063B000000A44F004040827009203E008224FF08A
:1063C000000A0092C4F30252022A05D059F804CB05
:1063D0000021032A08D009E009F1070121F0070292
:1063E000F2E802C1914605E01FFA8CFC042A01D1B3
:1063F0000CF0FF0C4FF00008220728D5702806D0BB
:10640000009B83F0100353EA0A0305D00EE04022FC
:106410008DF80420012208E05CEA010206D0302257
:106420008DF804208DF8050002229046009B83F031
:10643000080353EA0A030AD15CEA010201D16207A8
:1064400005D530228DF804204FF001087F1E582812
:1064500004D034A003900EA802900DE036A0F9E716
:1064600053466046009AF9F71DFF84460398825C04
:106470000298401E029002705CEA0100F0D102987E
:1064800006A9081A00F1200A600702D524F4803416
:1064900000E00127574502DDA7EB0A0000E00020DD
:1064A00000EB0A01009005984144401A0590E00372
:1064B00006D45B462146179A059800F0B6F90544C4
:1064C000002706E001A85A46C05D179990476D1C49
:1064D0007F1C4745F6DBE0030CD55B462146179A47
:1064E000059800F0A2F9054404E030205A461799B7
:1064F00090476D1C0099481E00900029F5DC08E0CB
:10650000029802995A460078491C029117999047BF
:106510006D1CBAF10001AAF1010AF1DC65E100008D
:106520000928010030313233343536373839616269
:10653000636465660000000030313233343536372D
:1065400038394142434445460000000000F05BF901
:106550000544761C307800287FF4ECAD19B028464D
:1065600000F04EB9620700D4062709F1070222F0B5
:10657000070CFCE80223E14603F000485FEA080C40
:1065800002D00FF2702C0DE05FEA045C02D50FF22E
:10659000682C07E05FEAC47C02D00FF2602C01E0B7
:1065A000AFF2700C4FF0FF3823F00043CDF850C02D
:1065B00065280CD006DC452809D046281DD0472880
:1065C0003DD13DE0662818D067287ED138E0002113
:1065D000112F01DB112000E0781CCDE9000106A994
:1065E0000EA8FFF7E9FCDDE90F010E9A03910021E7
:1065F000009207F1010A04914DE04FF0004000972E
:10660000CDE9011006A90EA8FFF7D6FCDDE90F02BF
:1066100003920E9B11990022DDF80CA000930492C6
:1066200011B9791C00EB010AB7EB0A0004D4C0F1E0
:10663000FF3007F1010A0490AAEB0700019044E043
:10664000012F00DA01270021112F01DD112000E0C8
:106650003846CDE9000106A90EA8FFF7ADFCDDE93B
:106660000F010E9A0391002104910092BA4621076E
:106670000CD40399514500DA8A46BAF1010F05DDC1
:10668000009AAAF10101515C302908D0B84202DA1F
:1066900010F1040F06DA0121CDE9011015E0AAF18D
:1066A0000101E9E7002805DC049901440491AAEB03
:1066B000000102E0411C514500DD8A460499401A60
:1066C000401C01904FF000400290200704D4019834
:1066D000504501DBCDF8048000208DF84F00029872
:1066E0000DF14F07B0F1004F25D02B200E900298EE
:1066F0004FF0020800280CDA404202902D200E9044
:1067000007E00A210298F9F74CFE3031029007F8B1
:10671000011DB8F10001A8F10108F2DC029800287F
:10672000EFD1791E0E980870307800F0200040F00C
:10673000450007F8020D12A8C01B00F107081498C5
:10674000007800B1012000EB0A01019801EBE07133
:1067500005984144401A401E0590E00306D45B466C
:106760002146179A059800F060F8054414980078BF
:1067700018B15A46179990476D1CE00324D55B4623
:106780002146179A059800F050F805441CE004983B
:10679000002807DBDDE90301884203DD0098405C47
:1067A000179901E0179930205A469047049805F14F
:1067B0000105401C04900198401E019004D12E2038
:1067C0005A46179990476D1CBAF10001AAF1010AC7
:1067D000DDDC05E017F8010B5A46179990476D1C50
:1067E000B8F10001A8F10108F4DC5B462146179AD4
:1067F0000598ABE62D0000002B00000020000000F3
:1068000030BCBDE8C08F2DE9F041044600251E468E
:106810001746880404D405E039462020B0476D1C93
:10682000641EF9D52846BDE8F0812DE9F041044603
:1068300000251E469046C80301D5302700E02027DA
:10684000880404D505E041463846B0476D1C641EF7
:10685000F9D52846BDE8F08113B54FF6FF73012244
:1068600069460248FDF7DAFA00981CBD18100020AE
:106870001CB50F4A01789279914201D0FF2913D1BA
:106880004178032910D1817840290DD1C188ADF814
:106890000010062100F04DF8ADF80400022201A915
:1068A0006846F9F75EFD08B100201CBD01201CBD43
:1068B000820100201CB50E4A01789279914213D1D1
:1068C0004178062910D1817840290DD1C188ADF8D1
:1068D0000010062100F02DF8ADF80400022201A9F5
:1068E0006846F9F73EFD08B100201CBD01201CBD23
:1068F00082010020FBF786FBFEF7A5FBFDF7D2FC2B
:10690000FDF754FCFDF7DCFBFDF7EAFDFDF762FE49
:10691000FDF77EFEFDF718FDFDF778FDFDF740FD64
:10692000FDF734FE00F02CF8FDF776FC00F03AF8A5
:10693000FEE770B504464FF6FF7000224AF20105EB
:106940000DE0A35C58400023C60702D085EA500042
:1069500000E040085B1C082BF6DB521C92B28A4216
:10696000EFD370BD10B5EFF3058111B16FF00504E1
:1069700003E0002408B101F043F8204610BD0000F8
:10698000EFF3058010B16FF005007047044801680F
:1069900011B14FF0FF3070470121016000207047B6
:1069A000F401002010B5EFF3058010B16FF0050081
:1069B00010BD08480168012902D04FF0FF3010BD1A
:1069C000054A002182F8141D0221016001F080F8BF
:1069D000002010BDF40100200BE000E0F8B51446E3
:1069E0004FF00005EFF3058212BB08B301B3A4B169
:1069F000D4E9023263B1502A1AD32269C2B167695D
:106A000000FB01F6B74213D3009501F090F907E0BF
:106A100072B9226962B9626952B9002201F066F95D
:106A2000050005D00CB1216800E0002100F0B2FFA4
:106A30002846F8BD2DE9FF410B464FF00005EFF366
:106A40000581039549BB40B38027182100244AB330
:106A5000166806B1344696691EB13146761E382E48
:106A600002D21679F60703D0002004B0BDE8F08109
:106A7000566906B1B708D2F808C0BCF1000F0DD0B6
:106A8000D5685C2D18D312693AB136B18DE806107D
:106A90003A46214601F026FC03900DE0D6685EB927
:106AA00012694AB903AACDE90012BAB2214601F02F
:106AB000E9FB012800D003950398D6E70349024873
:106AC0000968016070470000A001002080000020DC
:106AD00003490248C968016070470000980100201E
:106AE0000000002003490248096901607047000066
:106AF0009C010020000000200648054942690A6008
:106B000082694A60C2698A60006AC8607047000092
:106B1000CC1300200000002038B50546A0211D48F8
:106B2000F9F70DFC688869791A4C6A7840BA00292F
:106B30002ED07D292CD8184B9B79237062704A0087
:106B4000A2700022ADF800206B46E21C00F094FD1C
:106B500000281DD0BDF80000C01C81B22046FFF700
:106B6000E8FEBDF8001001222144C870BDF80010F5
:106B7000000A21440871BDF800002021401D85B2A3
:106B80000648FBF73CF92A4621460548FDF7A2F9DD
:106B900038BD00002C1300208201002000040048B2
:106BA000940F00202DE9F05F0546A0217348F9F706
:106BB000C6FB688895F8018047BAA88844F240026D
:106BC00045BA6F486D4CB91A00264FF0060A4FF0CF
:106BD000080B00F102094FF0020E974273D004DC5B
:106BE000303107D0012909D109E011293ED02029EF
:106BF000F9D15FE0A9F8065000F0A4FDA0E0691EFD
:106C0000072933D84F46A9F8085000F09BFDB87902
:106C1000207084F80180A6701120E07026716571E3
:106C200051462046FFF785FEA071000AE0715D46DF
:106C3000012220215348FBF7E2F82A462146524818
:106C4000FDF748F90A20FFF78DFE3889FEF7ACF909
:106C50004EA42046F9F77EFB82B2642321464A48BF
:106C6000FDF7DCF800F0AEB800F07EBD05804E48C0
:106C70004C494E4B026825B1012D08D0022D0ED093
:106C80005EE0D663006806640120187005E0D663F4
:106C90000068066483F800E00120087050E01E7070
:106CA0000E709FED430A434981ED000AD6630068E8
:106CB000066445E000EE105A3F48B8EE400A80ED09
:106CC000020A3DE0FFE7A5F5AA41993902D0113942
:106CD0002BD035E099F80600207084F80180A6706A
:106CE000E7702671657151462046FFF722FEA071BC
:106CF000000AE0715D46012220212248FBF77FF85F
:106D00002A4621462048FDF7E5F83220FFF72AFE03
:106D1000BFF34F8F29480168294A01F4E06111430C
:106D20000160BFF34F8F00BFFDE72222A9F80620C4
:106D3000A9F808E006807046FEF736F9FEF76AF813
:106D400099F80600207084F80180A670E77026711B
:106D5000657151462046FFF7ECFDA071000AE07115
:106D60005D46012220210748FBF749F82A462146C3
:106D700000F02DB80448FDF7ADB800002C1300203A
:106D80008001002000040048940F00204E65772009
:106D90006261756472617465206170706C696564AC
:106DA0000D0A000018010020200E00202401002000
:106DB0000000000010000020841200200CED00E014
:106DC0000400FA0530BCBDE8C05FFFF74DBF30BC22
:106DD000BDE8C05FFFF7CEBF2DE9F041134C0F4671
:106DE0000546E6682068001D00F0D6FC681C07D147
:106DF00037B12168BDE8F0410D48091D00F01CBD08
:106E000020683544B5424560216805D2A06BBDE8D5
:106E1000F041091D00F0F8BC606B091D00F0F4FCA6
:106E2000A06A854200D2A562BDE8F081A4010020DD
:106E3000CC1800202DE9F041054600F009FD2D4C4D
:106E4000A068401CA06020682B4F10B1606930B36F
:106E50002BE02560A068012827D1002606EB8600DC
:106E600007EB800000F0C2FC761C382EF6D32348D6
:106E700000F0BCFC2148143000F0B8FC1F4828305A
:106E800000F0B4FC1D483C3000F0B0FC1B48503012
:106E900000F0ACFC194860631430A06305E0206882
:106EA000E96AC06A884200D82560606A401C606256
:106EB0006864E86A2169884200D9206100EB80009B
:106EC00007EB8000291D00F0B7FC00F0E1FC6069D1
:106ED00000280CD02068E96AC06A884207D20849B5
:106EE0004FF080500860BFF34F8FBFF36F8FBDE846
:106EF000F0810000A40100201C1400207C18002058
:106F000004ED00E038B500F0A3FC104C2068C8B9CF
:106F10000F4800F06BFC0E48143000F067FC0C4882
:106F2000E060143020610A4B0020F03B009003F138
:106F3000500210210A2000F0FAFE206010B105A1D5
:106F400000F028FDBDE8384000F0A2BCE0010020C0
:106F5000D0190020546D72510000000030B4026C52
:106F60000B46002A0BD0C1681144C1608468A1425D
:106F700001D30168C16030BC1846F9F7C7B930BC0D
:106F800070472DE9F041856B174604460026026CD8
:106F900082B1C7B1E068F9F7B9F9E168206C091A64
:106FA000E1602268914202D2A168081AE060022FD3
:106FB00016D017E02068A8B9A06801F037FA064695
:106FC0000020A0600EE06068F9F7A0F9216C60680D
:106FD00008446060A168884204D32068606001E0D2
:106FE00005B16D1E6D1CA5633046BDE8F08110B57E
:106FF000044690F8590058B101280CD002280FD04F
:10700000502080F31188BFF34F8FBFF36F8FFEE7DF
:10701000206B00F051FC2046BDE8104000F04CBC55
:1070200010BD00000F4842F21071420705D0C01D8C
:107030000C4A20F00700821A891A0B4A00230144E7
:10704000C2E900030839183A21F0070111604B60CA
:107050000B600B1AC0E9001393604FF000405360BF
:1070600050617047B020002010020020144E154CD3
:10707000A6F29C474FF08058DFF84C9012E000BF1A
:1070800000F0E6FBF068C568281D00F085FBA068ED
:10709000401EA0606068401E606000F0F9FB28465A
:1070A000FFF7A5FF60680028EAD138680128F9D900
:1070B000C9F80080BFF34F8FBFF36F8FF2E7000076
:1070C000B8180020A401002004ED00E070B51D46B2
:1070D000049C51B1C4F80020C4E90F0101212046ED
:1070E00000F058FE84F84C5070BD2460F4E70000B6
:1070F0002DE9F05F8846DDE90B9415468346910043
:107100009A460A9EA522206BF9F712F96FF0030147
:10711000206B01EB8501084420F00707780707D0B2
:10712000502080F31188BFF34F8FBFF36F8FFEE7BE
:107130000025B8F1000F0FD05FF00000221818F8FA
:10714000001082F8341018F8001011B1401C1028FB
:10715000F4D384F8435001E084F83450382E00D33F
:107160003726E662C4E91365201D00F04AFB04F1EE
:10717000180000F046FB2461C6F138006462A0618B
:10718000656584F8585052465946384600F05EFA14
:107190002060B9F1000F01D0C9F8004000F000B83C
:1071A00030BCBDE8C09F000030B5114900E0114679
:1071B0000A688242FBD34B685C18844203D1406862
:1071C00018444860084643681C18944209D1084C8A
:1071D000183C2468A24209D052681A4442600A68E6
:1071E00012680260814200D0086030BD0460F9E797
:1071F0001002002070B5002441600B4D00619142E7
:1072000006D8D11A8269914206D2011D286907E089
:107210009A4203D2994201D3012403E0011DE86898
:1072200000F0F2FA204670BDE001002010B50446DF
:1072300000F00EFBA06B28B15FF0000400F028FB0B
:10724000204610BD0124F9E730B589B03C4D6EE011
:107250000498002806DADDE90601059A90470498AB
:10726000002864DB069C606910B1201D00F094FAD0
:1072700003A800F0D7F8024604980A2857D2DFE89E
:1072800000F00505052D334A05052D3394F8280037
:1072900040F0010084F828000599A069059B01448D
:1072A0002046FFF7A7FF68B3216A2046884794F875
:1072B000280040073BD5002000900598A1690023D5
:1072C00042181946204601F0BBF9D8B9502080F386
:1072D0001188BFF34F8FBFF36F8FFEE714F8280FAD
:1072E00020F00100207022E094F8280040F0010016
:1072F00084F828000598A06128B18118134620461B
:10730000FFF778FF13E0502080F31188BFF34F8F11
:10731000BFF36F8FFEE794F82800810703D420465F
:1073200000F0CAFA03E020F0010084F828000022EF
:1073300004A9286800F082FE002889D109B030BD78
:10734000E00100202DE9FC410F46054600F004FC59
:1073500001A800F067F80446019818B101F0DEF8C2
:10736000BDE8FC81254EAFB130690068D0B300277D
:10737000291B3A46306800F021FB01F0CFF80028C5
:10738000EED11F494FF080500860BFF34F8FBFF31D
:107390006F8FE5E7A542EBD801F0C0F8F06827460B
:1073A000C068C468201D00F0F7F994F82800410770
:1073B00019D5A0692B4641193A462046FFF71AFF16
:1073C000A8B100200346014600902A46204601F05D
:1073D00037F960B9502080F31188BFF34F8FBFF3A6
:1073E0006F8FFEE707E020F0010084F82800216A93
:1073F00020468847B4E70127BAE70000E0010020F3
:1074000004ED00E00648416B096829B1416BC96889
:10741000C9684968816270474FF0FF31FAE70000A0
:10742000A401002070B5054600F096FF064E044604
:10743000B068844203D200F009F8012000E0002087
:1074400028602046B46070BDE0010020F8B5194DF9
:1074500020E0C068C4680668201D00F09DF9216A1C
:107460002046884794F82800400713D5A069304487
:10747000B04206D924616060211DE86800F0C4F9BB
:1074800008E000200346014600903246204601F005
:10749000D7F838B1E86801680029DAD12969C5E967
:1074A0000310F8BD502080F31188BFF34F8FBFF356
:1074B0006F8FFEE7E001002008484068401C4FF055
:1074C000500080F3118804D0BFF34F8FBFF36F8F4C
:1074D000FEE7BFF34F8FBFF36F8FFEE71802002068
:1074E000074CE068016841B1C0680021D0F8000095
:1074F000FFF728FFFFF7A8FEF3E701210020F7E7D9
:10750000E00100202DE9F041044600F0A1F994F9D2
:10751000455004F1240609E0606A48B1304600F0A5
:10752000C5FF08B100F09AFA6D1E6DB2002DF3DCB4
:107530004FF0FF3684F8456000F0AAF900F088F9B2
:1075400094F9445004F1100709E0206948B1384625
:1075500000F0ACFF08B100F081FA6D1E6DB2002D95
:10756000F3DC84F84460BDE8F04100F091B900001C
:107570002DE9F0410546002700F0EEFA324E306862
:1075800008B9FFF74FFD706905424ED1C5B3083504
:1075900068070ED005F00700C0F108000544680731
:1075A00007D0502080F31188BFF34F8FBFF36F8F48
:1075B000FEE72DB37068854237D82348183001465E
:1075C0000C6801E020460C466168A94202D221689D
:1075D0000029F7D131688C4227D007682168016003
:1075E00060680837411B10290FD96019420708D07D
:1075F000502080F31188BFF34F8FBFF36F8FFEE7EA
:1076000013E041606560FFF7CFFD61687068401A64
:107610007060B268904200D2B0607069014300208F
:10762000C4E90001F068401CF06000F077FF7807C3
:1076300007D0502080F31188BFF34F8FBFF36F8FB7
:10764000FEE73846BDE8F081F801002010B5031FC1
:107650004FF080741C601B1F21F001011960191F7D
:10766000044B0B6014390A60091F6FF002024438A2
:107670000A6010BDB97400082DE9F0479A4600234E
:10768000DFF8BC904FE000254FEA090606EBC5077E
:1076900036F83540BF78A0422744BFB24AD3B8423B
:1076A00048D2041B1FFA84FC3C1AA4B2A14200D2A7
:1076B0000C4609EBC5056F68ED7875B300251AE037
:1076C0000CEB0506B6B24FEA560846F3000657F82B
:1076D0002880761C02D04FEA184601E01FFA88F68F
:1076E0004FEA162802F803805B1C9BB2D6545B1C41
:1076F0006D1C9BB2ADB2A542E2D310E00CEB0506C7
:1077000037F816604FEA162802F803805B1C9BB21C
:10771000D6545B1C6D1C9BB2ADB2A542EED3204487
:10772000091B80B289B20029ADD1AAF8003001202E
:10773000BDE8F0876D1C0B2DA8D30020F8E70000F2
:107740002801002010B5064C01212046F9F7E0FA87
:107750002046BDE8104005220249F9F73BBB000076
:1077600000F803088201002010B54FF48074214610
:107770000748F8F7E4FD07480068016841F0100188
:1077800001602246BDE8104001490248FCF7F0BA0A
:107790002C110020940F0020D0E9013201699A6079
:1077A000D0E901235A604A68824201D182684A6066
:1077B000002202610868401E0860086870470000E7
:1077C000034B036003F15C00086080201060704789
:1077D000F8190020044B036003F15C0008604FF4CB
:1077E0008070106070470000541C002000F10801F8
:1077F0004FF0FF32C0E90112C16001610021016058
:10780000704700210161704730B50B685A1C02D0E7
:1078100000F1080202E0026904E02246546825688B
:107820009D42FAD953684B6099608A605160086143
:107830000168491C016030BD42684A6093688B60F2
:1078400093685960916008610168491C0160704744
:10785000502080F31188BFF34F8FBFF36F8F0A4919
:107860004868401C486001280CD10848006810F0A6
:10787000FF0F07D0502080F31188BFF34F8FBFF365
:107880006F8FFEE7704700001802002004ED00E053
:107890000849486828B1401E486001D180F311882A
:1078A0007047502080F31188BFF34F8FBFF36F8F65
:1078B000FEE700001802002070B500282AD0164DFF
:1078C000A0F1080460686969084207D1502080F37C
:1078D0001188BFF34F8FBFF36F8FFEE722683AB175
:1078E000502080F31188BFF34F8FBFF36F8FFEE7F7
:1078F0008843606000F030F9606869680844686037
:107900002046FFF751FC2869401C2861BDE8704003
:1079100000F004BE70BD0000F80100204FF0E02030
:1079200000210161816105494FF47A720968B1FB58
:10793000F2F1491E41610721016170477400002086
:1079400010B5F8F789FC114910280ED300F1E0209A
:1079500090F8F0030A78904207D2502080F3118803
:10796000BFF34F8FBFF36F8FFEE709480068896848
:1079700000F4E060884207D9502080F31188BFF3FB
:107980004F8FBFF36F8FFEE710BD0000180200207D
:107990000CED00E010B5084B002200BF53F8324058
:1079A0001CB1521C082AF9D310BD43F8321003EB66
:1079B000C201486010BD0000DC13002070B5154600
:1079C0000E460446FFF744FF94F944100020491C7A
:1079D00001D184F8440094F94510491C01D184F880
:1079E0004500FFF755FFA06B28B92A46314604F140
:1079F000240000F051F82046BDE87040FFF782BD3A
:107A000010B5020014D00F48006B38B1502080F33D
:107A10001188BFF34F8FBFF36F8FFEE700F09CF824
:107A200000211046FFF7D8F900F078FD002807D1B3
:107A300005494FF080500860BFF34F8FBFF36F8F41
:107A400010BD0000A401002004ED00E002490A6A14
:107A50000260C96841607047A4010020014901200B
:107A6000C8617047A401002010B50C4650B1094907
:107A700009681831FFF7C8FE2046BDE81040012113
:107A8000FFF7AAB9502080F31188BFF34F8FBFF3DF
:107A90006F8FFEE7A401002070B514460D4668B153
:107AA0000A4909681831FFF7C7FE0CB14FF0FF35DE
:107AB00021462846BDE87040FFF78EB9502080F37C
:107AC0001188BFF34F8FBFF36F8FFEE7A401002033
:107AD00030B587B00024039405AA04A903A8049430
:107AE000FFF76EFEDDE903010094CDE901100023EC
:107AF00015A11748059A00F0F5FB164D0028E8621D
:107B00001FD000F06DFD012809D0401C19D1502074
:107B100080F31188BFF34F8FBFF36F8FFEE75020C4
:107B200080F31188BFF34F8FBFF36F8F4FF0FF309B
:107B3000A86201206861EC6007B0BDE8304000F049
:107B400045B807B030BD000049444C450000000076
:107B50006D700008A40100200248016B491C0163FC
:107B600070470000A4010020164810B5016B11B148
:107B70000121C16110BD0021C1610169124A01E00A
:107B8000B9B1491E01EB810352F82330002BF7D025
:107B900001EB810302EB830202F1080453685B6886
:107BA0005360A34201D15B685360DA6802600161EF
:107BB00010BD502080F31188BFF34F8FBFF36F8F3C
:107BC000FEE70000A40100201C1400201CB537486B
:107BD0000168374A914207D1502080F31188BFF3E2
:107BE0004F8FBFF36F8FFEE700683149491E88420F
:107BF00007D1502080F31188BFF34F8FBFF36F8FF1
:107C0000FEE72C4908780190FF20087008788DF86D
:107C100000009DF800009DF8002000F0F000904268
:107C200007D0502080F31188BFF34F8FBFF36F8FC1
:107C3000FEE79DF80000204C00F050002070072067
:107C4000A06005E09DF8002052008DF80020401E45
:107C50009DF800201206F5D4A060032807D050201C
:107C600080F31188BFF34F8FBFF36F8FFEE74FF4A0
:107C70004070A060019808700C482030016841F401
:107C800070010160016841F070410160FFF746FE3C
:107C900000206060F8F7A8FA0848016841F0404108
:107CA0000160F8F78DFA00201CBD000000ED00E037
:107CB00071C20F4100E400E01802002034EF00E040
:107CC00010B5502080F31188BFF34F8FBFF36F8F33
:107CD00000F048FB18B104494FF0805008600020C4
:107CE00080F3118810BD000004ED00E0F8B51746E0
:107CF0000E46050013D005FB06F05030FFF738FCA8
:107D000004000AD0002084F8460004F150023B46EB
:107D1000314628460094FFF7D9F92046F8BD502097
:107D200080F31188BFF34F8FBFF36F8FFEE738B535
:107D3000049D18B153B1CAB181B120E0502080F345
:107D40001188BFF34F8FBFF36F8FFEE7502080F392
:107D50001188BFF34F8FBFF36F8FFEE7502080F382
:107D60001188BFF34F8FBFF36F8FFEE739B15020FB
:107D700080F31188BFF34F8FBFF36F8FFEE750245E
:107D80001C46012384F846302B460094FFF79EF9E9
:107D9000204638BD70B50D46040025D0FFF758FDCC
:107DA000D4E90F20216802FB0011A1600021A1632A
:107DB000216861600A46D4E90F01401E00FB0121E1
:107DC000E16021464FF0FF3001F8440F487004F1A4
:107DD00010008DB1FFF70AFD04F12400FFF706FD46
:107DE000FFF756FD012070BD502080F31188BFF3CE
:107DF0004F8FBFF36F8FFEE721690029F0D000F0AD
:107E000055FB0028ECD004494FF080500860BFF3C8
:107E10004F8FBFF36F8FE3E704ED00E02DE9FF47DD
:107E200082B01D468A464FF00008040003D0BAF124
:107E3000000F08D011E0502080F31188BFF34F8F5E
:107E4000BFF36F8FFEE7206C38B1502080F31188AC
:107E5000BFF34F8FBFF36F8FFEE7022D0AD1E06BA8
:107E6000012807D0502080F31188BFF34F8FBFF354
:107E70006F8FFEE700F062FA3F4F4FF000094FF0BE
:107E8000805648B9049838B1502080F31188BFF368
:107E90004F8FBFF36F8FFEE7FFF7DAFCA06BE16B4C
:107EA000884207D3022D05D00498D0B1B8F1000F55
:107EB0001AD01EE02A4651462046FFF762F8616A52
:107EC00019B104F1240000F0F1FA20B13E60BFF3D3
:107ED0004F8FBFF36F8FFFF7DBFC012006B0BDE8CB
:107EE000F087FFF7D5FC22E06846FFF7AFFD4FF0C3
:107EF0000108FFF7CDFCFFF72FFEFFF7A9FC94F96F
:107F00004400401C01D184F8449094F94500401C81
:107F100001D184F84590FFF7BBFC04A9684600F046
:107F200077F930B12046FFF7EDFA00F0F7FA0020BC
:107F3000D4E7FFF78DFCA06BE16B884213D1FFF70C
:107F4000A7FC04F110000499FFF78EFD2046FFF70F
:107F5000D9FA00F0E3FA00289ED13E60BFF34F8FBC
:107F6000BFF36F8F98E7FFF793FC2046FFF7CAFA3D
:107F700000F0D4FA90E7000004ED00E02DE9F047AE
:107F80001F4690468946040003D0B9F1000F08D07F
:107F900011E0502080F31188BFF34F8FBFF36F8F34
:107FA000FEE7206C38B1502080F31188BFF34F8F6B
:107FB000BFF36F8FFEE7022F0AD1E06B012807D0D5
:107FC000502080F31188BFF34F8FBFF36F8FFEE710
:107FD000FFF7B6FC5020EFF3118680F31188BFF352
:107FE0004F8FBFF36F8FA06BE16B884206D3022FD8
:107FF00004D0002086F31188BDE8F08794F945503D
:10800000A06B3A4649462046FEF7BBFF681C04D0E9
:108010006D1C84F845500120ECE7606A0028FAD016
:1080200004F1240000F042FA0028F4D0B8F1000F67
:10803000F1D00121C8F80010EDE700002DE9F74765
:10804000002683B08A46040003D0BAF1000F08D09E
:1080500011E0502080F31188BFF34F8FBFF36F8F73
:10806000FEE7206C38B1502080F31188BFF34F8FAA
:10807000BFF36F8FFEE700F061F9DFF8F4804FF097
:1080800000094FF0805748B9059838B1502080F367
:108090001188BFF34F8FBFF36F8FFEE7FFF7D8FB59
:1080A000A56BC5B151462046FEF758FF6D1EA5636E
:1080B000206950B104F1100000F0F8F928B1C8F8B7
:1080C0000070BFF34F8FBFF36F8FFFF7E1FB01200D
:1080D00006B0BDE8F087059808B11EB106E0FFF7CD
:1080E000D7FB27E06846FFF7B1FC0126FFF7D0FB7E
:1080F000FFF732FDFFF7ACFB94F94400401C01D1BF
:1081000084F8449094F94500401C01D184F84590CE
:10811000FFF7BEFB05A9684600F07AF80028204664
:108120000AD0FFF7EFF900F0F9F92046FFF77EF8E3
:108130000028B3D00020CBE7FFF778F890B104F126
:1081400024000599FFF790FC2046FFF7DBF900F0CB
:10815000E5F90028A2D1C8F80070BFF34F8FBFF334
:108160006F8F9BE72046FFF7CDF900F0D7F995E731
:1081700004ED00E02DE9F04790468946040003D065
:10818000B9F1000F08D011E0502080F31188BFF33F
:108190004F8FBFF36F8FFEE7206C38B1502080F314
:1081A0001188BFF34F8FBFF36F8FFEE7FFF7C8FB58
:1081B0005020EFF3118680F31188BFF34F8FBFF388
:1081C0006F8FA76BF7B194F9445049462046FEF7EC
:1081D000C5FE7F1EA763681C04D06D1C84F8445044
:1081E000012010E020690028FAD004F1100000F00E
:1081F0005DF90028F4D0B8F1000FF1D00121C8F8E2
:108200000010EDE7002086F31188BDE8F08700003C
:108210002DE9F0410C46050011D0C4B1FFF718FB61
:10822000174BDA686E682068911B471C17D02F68BF
:108230001B6A9F4219D0964217D8012410E05020A3
:1082400080F31188BFF34F8FBFF36F8FFEE750208D
:1082500080F31188BFF34F8FBFF36F8FFEE70024C9
:10826000FFF716FB2046BDE8F081884205D9401A89
:1082700020602846FFF7EAFBF1E700202060DCE7FA
:10828000A40100202DE9FF5F8346DDE90E879946B2
:1082900016468A469000FFF76BF905001CD05C205B
:1082A000FFF766F9040014D00020256384F8590014
:1082B000CDE90240CDE900874B463246514658464B
:1082C000FEF716FF2046FEF7B5FD012004B000F0D2
:1082D00006B82846FFF7F0FA4FF0FF30F6E730BC5B
:1082E000BDE8C09FF0B585B0DDE90B640A9DA6B17D
:1082F000DCB15C2700972663022684F859600026CB
:1083000004AFCDE90246CDE90057FEF7F1FE204665
:10831000FEF790FD049805B0F0BD502080F3118861
:10832000BFF34F8FBFF36F8FFEE7502080F31188AC
:10833000BFF34F8FBFF36F8FFEE700000548416921
:1083400019B1006B18B1002070470120704702205E
:1083500070470000A40100200148C0687047000079
:10836000A40100202DE9F0412E4C0027206B28B1FC
:10837000A069401CA0613846BDE8F081E668761C23
:10838000E66013D1606B006838B1502080F311882B
:10839000BFF34F8FBFF36F8FFEE7606BA16B61631D
:1083A000A063206A401C2062FFF72CF8A06ADFF867
:1083B0007880864209D3606B0068A0B1606BC068AA
:1083C000C5686868864211D2A0622068C06A00EB66
:1083D000800158F82100012800D90127E069002810
:1083E000C9D00127C7E74FF0FF30EDE7281DFFF7A1
:1083F000D3F9A86A18B105F11800FFF7CDF9E86ABA
:108400002169884200D9206100EB800108EB8100DE
:10841000291DFFF711FAE86A2168C96A8842CAD3A0
:108420000127C8E7A40100201C14002070B5040037
:108430004FF0000133D01B4D2868844207D05020F4
:1084400080F31188BFF34F8FBFF36F8FFEE7206D6E
:1084500038B1401E2065E36CE26A9A421FD040B1F9
:108460001DE0502080F31188BFF34F8FBFF36F8F53
:10847000FEE7201DFFF790F9E06CE062C0F13800E4
:10848000A061E06A2969884200D92861064900EBA9
:10849000800001EB8000211DFFF7CEF90121084685
:1084A00070BD0000A40100201C14002070B5C0683D
:1084B000C46854B104F118000646FFF76DF9144D75
:1084C000286B50B13146134815E0502080F31188D5
:1084D000BFF34F8FBFF36F8FFEE7201DFFF75CF9EF
:1084E000E06A2969884200D928610B4900EB8000C5
:1084F00001EB8000211DFFF79FF9E06A2968C96A36
:10850000884202D90120E86170BD002070BD0000E2
:10851000A4010020A41800201C1400202DE9F0471D
:108520002C4D00242746286B38B1FFF791F9286BB2
:10853000401E2863286B40B146E0502080F311882C
:10854000BFF34F8FBFF36F8FFEE7A968224E012064
:10855000D1B3A6F5916980463068E0B1F068C4688F
:1085600004F11800FFF718F9201DFFF715F9E06A6C
:108570002969884200D9286100EB800109EB81005C
:10858000211DFFF759F9E06A2968C96A8842E3D3D7
:10859000C5F81C80E0E70CB1FEF734FFAC694CB1C4
:1085A0004FEA0806FFF7DEFE00B1EE61641EF9D166
:1085B0000020A861E86938B1084901273807086038
:1085C000BFF34F8FBFF36F8FFFF762F93846BDE8F7
:1085D000F0870000A4010020A418002004ED00E0B2
:1085E00010B586B0FEF78EFC114C2068B8B10020A3
:1085F0000390049005AA04A903A8FFF7EBF8DDE9AE
:10860000032102208DE8070000230AA10B48059AE8
:10861000FFF768FE606010B106B0012010BD502069
:1086200080F31188BFF34F8FBFF36F8FFEE7000019
:10863000E0010020546D722053766300E17400085D
:108640002DE9FF411E46134602000A9D4FF000002F
:1086500016D0144C2768002F0FD0CDE900130292DA
:10866000062917DAFFF76AFE02284FF000030FD041
:10867000002269462068FFF7D1FB04B0BDE8F08115
:10868000502080F31188BFF34F8FBFF36F8FFEE749
:108690002A46EEE70023324669463846FFF76EFC6D
:1086A000EBE70000E0010020FC870008000000006C
:1086B00000000000000000000000000000020000B8
:1086C000300000000000000000000000D887000813
:1086D000000000000000000000000000000000009A
:1086E0000002000018000000000000000000000070
:1086F000BC8700080000000000000000000000002F
:10870000000000000002000008000000000000005F
:1087100000000000E48700080000000000000000E6
:10872000000000000000000000020000180000002F
:108730000000000000000000F087000800000000BA
:108740000000000000000000000000000002000027
:10875000180000000000000000000000C8870008AA
:1087600000000000840C0020500000008402002063
:10877000000A0000000000000000000001020304E5
:1087800006070809A0860100400D0300801A0600B4
:1087900000350C0040420F0080841E0000093D009F
:1087A00000127A000024F40000366E010048E8014F
:1087B000006CDC02000000000102030452656164E9
:1087C0005461736B303200007561727434383572E5
:1087D0007871756575650000526561645461736BED
:1087E0000000000053656E645461736B000000006C
:1087F0004D6F746F725461736B0000004869676855
:108800006573745461736B002888000800000020B1
:108810002802000040090008B08800082802002053
:1088200098490000AA5F0008014832010A19101C8B
:10883000D10B33093D6071FA4869120403104840B6
:108840001914DA801CE204694812480A130820E16E
:1088500013400213820115200240011A86081A10E3
:10886000081A88081A11081A8A08142040031A8C5A
:10887000081A50101A94081A51081A80081E5240FB
:10888000020198081A54081A9C081A56081AA008D7
:108890001758400801CC1322201B2522DC1301228B
:1088A0001202122207880619010AA5A51AAA018137
:040000050800018D61
:00000001FF
